:020000040800F2
:1000000060110020A1010008DD5A000881430008AA
:10001000D95A000829100008B1700008000000003B
:10002000000000000000000000000000F95E000871
:10003000C313000800000000915B0008296300085A
:10004000BB010008BB010008BB010008BB010008A0
:10005000BB010008BB010008BB010008BB01000890
:10006000BB010008BB010008BB010008BB01000880
:10007000BB010008D5120008BB010008BB01000845
:10008000BB010008BB010008BB010008BB01000860
:10009000BB010008BB010008BB010008BB01000850
:1000A000BB010008BB010008BB010008BB01000840
:1000B000F563000805640008BB010008BB010008E7
:1000C000BB010008BB010008BB010008BB01000820
:1000D000BB010008BB010008416D0008BB0100081E
:1000E000BB010008BB010008BB010008BB01000800
:1000F000BB010008BB010008BB010008BB010008F0
:10010000BB010008BB010008BB010008BB010008DF
:100110003D680008BB01000815640008256400085C
:10012000BB010008BB010008BB010008BB010008BF
:10013000BB010008BB010008BB010008BB010008AF
:10014000BB010008BB010008BB010008BB0100089F
:10015000BB010008BB010008BB010008BB0100088F
:10016000BB010008BB010008BB010008BB0100087F
:10017000BB010008BB010008BB0100080000000033
:10018000BB010008BB010008DFF810D000F08AFCBA
:1001900000480047657F0008AFF300806011002031
:1001A0000648804706480047FEE7FEE7FEE7FEE711
:1001B000FEE7FEE7FEE7FEE7FEE7FEE7E163000895
:1001C000890100082DE9F05F0546002092469B4614
:1001D00088460646814640241BE02846414647465D
:1001E000224600F024FB53465A46C01A914110D3D0
:1001F00011461846224600F00BFB2D1A67EB01084A
:100200004F4622460120002100F002FB17EB0009B7
:100210004E41201EA4F10104DFDC484631462A4647
:100220004346BDE8F09FD2B201E000F8012B491E21
:10023000FBD270470022F6E710B513460A46044683
:100240001946FFF7F0FF204610BD30B505462A4697
:100250000B4612F8010B13F8014B08B1A042F8D07D
:100260001CB1002802D06D1CF1E7284630BD10B546
:10027000044604E00B7800F8013B03B1491C521E10
:10028000F8D2204610BDCAB2401E10F8011F8A42A3
:1002900002D00029F9D100207047421C10F8011B40
:1002A0000029FBD1801A70470022CBB20178994215
:1002B00000D10246401C0029F8D1104670470000CA
:1002C0000FB400B58DB010A909900B9000914FF0BC
:1002D000FF300A9000200C900548069005480790D2
:1002E0006A4609A80F9900F0D9FA0DB05DF814FB21
:1002F000B9080008D70800082DE9FF5F1D464FF038
:10030000FF3BD5E9014691465F464FF00008A969D9
:100310007F1C01988847296A824688470028F6D1C1
:10032000BAF1FF3F0CD024F4C064002E19DD600642
:1003300014D5BAF12B0F09D0BAF12D0F0ED103E06D
:10034000584604B0BDE8F09F44F48064A9697F1C5E
:1003500001988847761E8246002E02DDBAF1300FE2
:1003600003D0B9F1000F26D032E0A969761E44F41B
:1003700000747F1C019888478246002E05DDBAF183
:10038000780F06D0BAF1580F03D0B9F1000F10D092
:100390001EE0B9F1000F02D0B9F1100F18D1A96910
:1003A000761E24F400747F1C019888478246102032
:1003B00002E0082000E00A20814609E008FB090865
:1003C000A969761E44F400747F1C01988847824610
:1003D000002E05DD4946504600F04BFA0028EDDAC4
:1003E000E96901988847A00502D46FF00100A8E7E9
:1003F000E00725D1600613D5600502D5C8F10000DD
:1004000000E0404629680A1D2A600968220501D5D6
:10041000087015E0220701D5088011E008600FE0A0
:100420002868011D29600068210502D580F8008038
:1004300006E0210702D5A0F8008001E0C0F80080A6
:1004400038467EE72DE9FE4F804681EA0300C00F63
:100450000C46009021F0004123F00045B8EB02006B
:10046000A94105D24046214690461C460B4602460D
:1004700023F00040104347D0270DC7F30A00C3F311
:100480000A510290401A019040286BDAC3F313001E
:1004900040F4801B0098924620B10023D2EB030A5F
:1004A00063EB0B0B01985946C0F14002504600F037
:1004B000AFF906460D4650465946019A00F0C7F975
:1004C00010EB08006141002487EA115284EAE773C7
:1004D0001A4340D0009A62B3019A012A4FEA0752A8
:1004E00015DC001B61EB02014FF0004202EA0752EB
:1004F000CDE90042001C41F5801132462B4600F048
:1005000041FA03B0BDE8F08F40462146F9E7001BF1
:1005100061EB0201001C41F5801300185B412018BB
:10052000A2F5001747EB030140EAD570B6196D41FB
:1005300011E06D084FEA360645EAC0754FEA0752EA
:10054000001B61EB0201001C41F5801149084FEAD4
:1005500030000019514132462B4603B0BDE8F04F40
:1005600000F001BA0098012240000023D0EB020203
:1005700063EBE073009821464FEAE074B8EB0000AB
:1005800061EB0401E9E783F000435BE781F00041A0
:1005900058E72DE9FE4F81EA030404F0004421F0FE
:1005A000004100944FF0000B23F0004350EA010497
:1005B0005ED052EA03045BD0C3F30A54C1F30A5578
:1005C0002C44A4F2F3340194A0FB0254C1F31301B0
:1005D00041F48011C3F3130343F4801301FB02447D
:1005E00000FB034E840A970A44EA815447EA835782
:1005F000A4FB076802958D0A05FB07854FEA932C3B
:1006000004FB0C542705029D4FEA065847EA1637AB
:10061000B5EB08056EEB070C870E920E47EA8117C3
:1006200042EA8312A7FB0201B6EB0B0164EB000464
:100630002B0D43EA0C335E1844EB1C50DA4651464E
:10064000E7FB0201C5F313044FEA0B3343EA1453EB
:100650004FEA0432019C43EA0603A4F10C0402941D
:10066000009CCDE900B400F08DF903B0BDE8F08F37
:1006700000200146F9E72DE9F04D81EA030404F07A
:10068000004B21F0004514464FF0000A23F00041D2
:1006900050EA050220D054EA01021DD0C5F30A57E2
:1006A0000246C5F31303C1F31300C1F30A5640F425
:1006B000801543F48013A7EB0608101BD64608F2FA
:1006C000FD3873EB050002D308F1010801E0921830
:1006D0005B41B8F1000F03DA00200146BDE8F08D60
:1006E00000204FF48011064684460EE0171B73EB82
:1006F000050705D3121B63EB050306434CEA010C07
:1007000049084FEA300092185B4150EA0107EDD1E9
:1007100052EA030012D082EA040083EA050108438A
:1007200005D0101BAB4106D20122002306E00022B7
:100730004FF0004302E06FF0010253101AEB060085
:100740004CEB085110EB0A0041EB0B01BDE8F04DFA
:1007500000F009B900F0004230F000400AD0C10DAD
:1007600001F56071C0F3160042EA0151C20840076A
:1007700011437047002001467047000030B5041E49
:1007800071F1000404DB4FF00044404264EB0101CE
:10079000141E73F1000405DB1C464FF00043524267
:1007A00063EB0403994208BF904230BD01F000435F
:1007B00030B421F0004150EA010206D00A0DA2F542
:1007C0006072C1F31301002A02DC30BC00207047C4
:1007D000440F44EAC104C100E01830BC00EBC25031
:1007E00000F08AB830B50B460146002020220124D3
:1007F00009E021FA02F59D4205D303FA02F5491BEF
:1008000004FA02F52844151EA2F10102F1DC30BD04
:10081000202A04DB203A00FA02F1002070479140C0
:10082000C2F1200320FA03F3194390407047202AB5
:1008300004DB203A21FA02F00021704721FA02F38A
:10084000D040C2F120029140084319467047202A47
:1008500006DBCB17203A41FA02F043EAE07306E0E8
:1008600041FA02F3D040C2F12002914008431946F8
:1008700070473A2800D2303820F02002412A01D3B4
:10088000A2F13700884201D34FF0FF3070470000DB
:10089000026811441378016018467047D16004491A
:1008A00051610449116200211161114600F012B931
:1008B00091080008C90A0008426842B1016811F8AD
:1008C000013B23B1521EC0E90012184670470121B6
:1008D000C160881E704742685AB1C368016843B955
:1008E00083688B4205D0491E521CC0E900120020CB
:1008F00070474FF0FF3070470029A8BF7047401C79
:10090000490008BF20F00100704710B4B0FA80FC25
:1009100000FA0CF050EA010404BF10BC704749B162
:10092000CCF1200421FA04F411FA0CF118BF0121D2
:1009300021430843A3EB0C01CB1D4FEA00614FEAB2
:10094000102042BF002010BC704700EBC350104481
:100950000029A4BF10BC7047401C490008BF20F00C
:10096000010010BC704710B5141E73F1000408DAC2
:10097000401C41F1000192185B411A4301D120F063
:10098000010010BD2DE9F04D92469B4611B1B1FA20
:1009900081F202E0B0FA80F220329046FFF738FF91
:1009A00004460F4640EA0A0041EA0B0153465A4604
:1009B000084313D0114653EA010019D0C8F1400290
:1009C0005046FFF734FF05460E465046594642460C
:1009D000FFF71EFF084305D0012004E020463946FA
:1009E000BDE8F08D0020054346EAE0762C4337430E
:1009F0000A986305E40AA0EB08000022FD0A44EA15
:100A000047540A3002D500200146E9E701051019D4
:100A10006941DDE9084500196941BDE8F04DA2E7EB
:100A20000EB5C10F80EAE0700844CA07002140F209
:100A300033438DE80E000A460B46FFF7A3FF03B0D1
:100A400000BDC1F30A52C1F3130140F2FF3341F478
:100A500080119A4202DA00200146704740F2334387
:100A60009A42A2F2334202DC5242FFF7E0BEFFF7A5
:100A7000CFBE000030B5041E71F1000404DB4FF05E
:100A80000044404264EB0101141E73F1000405DBD5
:100A90001C464FF00043524263EB04038B4208BFF5
:100AA000824230BD064C074D06E0E06840F001038D
:100AB00094E8070098471034AC42F6D3FFF768FB80
:100AC00098820008B8820008C0B24FF4F05100F0DC
:100AD00099B900002DE9F34F8BB04FF0000801F1F8
:100AE0000C000C464FF0010B46460DF1080A019030
:100AF0006269012101989047051E2DD0252D2CD02B
:100B0000216A8847C0B16269012101989047216A32
:100B100088470028F7D1411E62690198904700E09C
:100B2000761CA1690B988847216A88470028F7D16D
:100B3000E1690B988847DBE7A1690B98884707466E
:100B4000A84201D1761CD3E7E1690B9888477F1C46
:100B500002D1B8F1000F6FD047E1002762693D462E
:100B60003946019890472A2804D1626901210198E9
:100B700090470125DFF8889262690121019890472A
:100B8000A0F130010A290AD24F45E5DC07EB8701C5
:100B900000EB4107303FDFD445F01005ECE7E906F4
:100BA00001D46FF000476C280AD04C2814D0682874
:100BB00015D06A280DD074281CD07A281AD01DE0D0
:100BC00062690121019890476C2802D045F0040524
:100BD00014E045F002050DE045F020050AE06269E9
:100BE000012101989047682802D045F0080505E0EA
:100BF00045F400656269012101989047C4E90157F5
:100C000065283DD019DC58287AD00CDC452837D02F
:100C100004DC252826D0412831D131E046282FD0C8
:100C200047282CD12CE05B2877D0612828D0632876
:100C30007CD0642823D15AE0D1E06F2848D008DC6A
:100C400066281DD067281BD0692821D06E2816D1B0
:100C500027E0702845D0732868D0752847D07828B9
:100C60000DD14DE0A1690B988847054625283FF432
:100C700069AFE1690B9888476D1C3FF46AAFB4E037
:100C800023466A466FF001000B99AFF300809FE0A6
:100C900045F040006060A80723464FF0000236D4BC
:100CA0003EE0E8077FF447AF2068011D216000683F
:100CB000290501D506701BE7290701D5068017E72E
:100CC000A90703D5F117C0E9006111E706600FE736
:100CD00045F040006060A80723464FF0080216D494
:100CE0001EE040F60E0125EA0100606016E045F0C6
:100CF00040006060A80723464FF00A0207D40FE0C7
:100D000045F040006060A80708D5234610226FF028
:100D100001000B99AFF300805AE007E02346102250
:100D20006FF001000B99FFF7E7FA51E04FF000096F
:100D30004F464B46632802D05B2807D041E020791C
:100D4000C00601D40120A06001273AE062690121B8
:100D5000019890475E2805D14FF001096269494624
:100D600001989047216939B900210A46534643F852
:100D70002120491C0829FADBB0B3216969B9C117E0
:100D800000EBD16253110AEB830122F01F02821A99
:100D900001200B68904003430B60626901210198B8
:100DA00090475D28E8D1B9F1000F09D000205146E5
:100DB00051F82020D24341F82020401C0828F7DBBE
:100DC00002AB224600976FF001000B99AFF3008051
:100DD00000280CDA401C08D1BBF1000F05D04FF001
:100DE000FF300DB0BDE8F08FFFE74046F9E7E907B7
:100DF00001D108F1010806444FF0000B78E600002D
:100E0000CCCCCC0C7F2801D9002208E0064A02EBAA
:100E10005002C007127800D1120902F00F0201201F
:100E200090400840704700003881000870B58C1869
:100E300010F8015B15F0070301D110F8013B2A11EE
:100E400006D110F8012B03E010F8016B01F8016BDB
:100E50005B1EF9D12B0705D40023521E0DD401F8D7
:100E6000013BFAE710F8013BCB1A921C03E013F8A0
:100E7000015B01F8015B521EF9D5A142D8D30020D5
:100E800070BD000055494A6822F440324A604A6801
:100E900043681A434A600268526822F48072036809
:100EA0005A6002685368026943EA022203685A6082
:100EB0000268526822F0407203685A600268526801
:100EC00083681A4303685A600268926822F40062D9
:100ED00003689A6002689268C3681A4303689A605C
:100EE0003F4B826A9A4218D00268926822F0706280
:100EF00003689A6002689268836A1A4303689A607A
:100F00000268926822F0405203689A600268926810
:100F1000C36A1A4303689A600BE00268926822F081
:100F2000706203689A600268926822F04052036817
:100F30009A600268926822F0020203689A6002686E
:100F40009368027E43EA420203689A602022125CA0
:100F5000A2B10268526842F4006203685A600268F3
:100F6000526822F4604203685A6002685368426A19
:100F7000521E43EA423203685A6005E00268526832
:100F800022F4006203685A600268D26A22F4700296
:100F90000368DA620268D36A828B521E43EA025205
:100FA0000368DA620268926822F4007203689A6049
:100FB0000268936890F8302043EA422203689A60FE
:100FC0000268926822F4806203689A6002689368FB
:100FD000426943EA822203689A6070470023014015
:100FE0000100000F10B504F01FFD01220749084859
:100FF00003F00CF99FED070B084880ED000B9FED07
:10100000080A084880ED010A10BD00000C0000200D
:10101000D80300200000000000000000B8010020FC
:1010200000000000500D002000BFFEE710B501F0E9
:10103000BDFA044615480068201A4EF66021884221
:1010400022D31248046080211148FFF7F3F80020F2
:101050001049088010A003F081FC642001F08AF997
:1010600011A10B48FFF7F1F858B91348007803288D
:101070000ADA11480078401C0F49087003F0F0FCB0
:1010800002E000200C49087010BD00005400002050
:10109000100500204C00002041542B514D54434F6B
:1010A0004E4E3F0D0A0000002B514D54434F4E4E03
:1010B0003A20302C330000005800002010B504F016
:1010C000AFFE044612480078844206D011480078EA
:1010D000401C104908700E4804700F480068401CFE
:1010E0000D4908600846006864280FD30948007855
:1010F000052803DB01200949087002E002200749A6
:1011000008700020034908700349086010BD000002
:10111000FD010020FE01002000020020FC01002053
:1011200070B50446012C05D1002010490870104903
:10113000087019E0C4B90F480578002000F0B8F82D
:10114000002000F019F8002000F028F8002000F03E
:1011500055F8002004F0C4FC01200449087004493B
:1011600008700448057000BF70BD000044000020F6
:10117000450000201801002010B504462CB10122C2
:101180000421054801F00CFA04E000220421024881
:1011900001F006FA10BD00000018024010B5044628
:1011A0002CB101220821054801F0FAF904E00022DF
:1011B0000821024801F0F4F910BD000000180240B7
:1011C00010B5044684B10C48007830B90120FFF70F
:1011D000D3FF0020FFF7E2FF0CE00020FFF7CCFF79
:1011E0000120FFF7DBFF05E00020FFF7C5FF00202F
:1011F000FFF7D4FF10BD00002401002010B5044605
:101200000CB1012000E0002002464FF400710248BA
:1012100001F0C6F910BD00000018024010B50446E8
:1012200034B1012000F020F8012000F02FF805E093
:10123000002000F019F8002000F028F810BD000090
:1012400010B50848007830B1012000F00DF80020FA
:1012500000F01CF805E0002000F006F8012000F086
:1012600015F810BDDD01002010B504460CB10120B9
:1012700000E0002002460421024801F091F90248F2
:10128000447210BD001002409008002010B50446C2
:101290000CB1012000E0002002460821024801F0C4
:1012A0007FF90248847210BD0010024090080020AF
:1012B00010B504462CB101220221054801F070F955
:1012C00004E000220221024801F06AF910BD00008A
:1012D0000018024010B5024800F0B6FE10BD000034
:1012E000B00400200146087810381823B0FBF3F250
:1012F0000848805CC865032A05D908686FF30900AF
:10130000001D886503E008686FF309008865886D33
:1013100070470000D4800008014600208A6A8B696B
:10132000CBB932B1012A0DD0022A03D0032A10D141
:101330000EE000BFCB6A03F08073B3F1807F00D171
:10134000012007E0CB6AB3F1C07F00D1012001E0AA
:1013500000E000BF34E08B69B3F5005F1AD132B111
:10136000012A07D0022A03D0032A11D10AE000BFC4
:1013700001200EE0CB6A03F08073B3F1807F00D1CF
:10138000012006E0CB6AB3F1C07F00D1012000E06C
:1013900000BF15E032B1012A05D0022A04D0032A89
:1013A0000CD103E000BF00BF012008E0CB6A03F0CE
:1013B0008073B3F1807F00D1012000E000BF00BF47
:1013C0007047704710B503F01BFB05F0E3F80020F1
:1013D000FFF76EFF0020FFF7CFFE0020FFF7DEFED5
:1013E00000200A4908600A4908600A49087001207B
:1013F0000949087000200949087004F0D7FC084921
:101400000870084600780749087010BD1C010020CC
:1014100020010020240100202501002026010020B9
:10142000270100202801002010B504F0C7FC044665
:101430005C480078844209D000205B4908605B4921
:10144000086001205A49087056480470002C52D197
:101450005848007830B10020FFF72AFF0020564995
:1014600008601FE05048006854490968884206D265
:101470000120FFF71DFF01204F49086012E04F488F
:1014800000684F490968084447490968884206D9F5
:101490000020FFF70DFF00204749086002E0002010
:1014A000414908604748007818B10020FFF788FEDE
:1014B00077E03E48006844490968884203D2012029
:1014C000FFF77EFE6DE00020FFF77AFE3E480068E1
:1014D0003E490968084435490968884261D80020B6
:1014E000324908603A48007808B9012000E000203D
:1014F0003749087055E00020FFF7DAFE00202E493A
:1015000008603048007818B10020FFF759FE48E025
:101510002748007820B3254800682E49096888428A
:1015200003D20120FFF74CFE3BE00020FFF748FE0E
:10153000284800682849096808441C490968884205
:101540002FD80020194908602148007808B90120E7
:1015500000E000201E49087000201549087020E0B6
:10156000124800681D490968884203D20120FFF72C
:1015700027FE16E00020FFF723FE184800681849F0
:10158000096808440949096888420AD800200749BF
:1015900008600F48007808B9012000E000200C49DD
:1015A000087010BD300100201C0100202001002027
:1015B00025010020440000202C0100209400002080
:1015C00098000020450000209C000020A000002082
:1015D00024010020AC000020B0000020A400002066
:1015E000A800002010B51048007868B10F480068C6
:1015F000052809D3002210210D4800F0D1FF00205A
:1016000009490870094908600A48006848280AD34F
:1016100000200849086001221021054800F0C0FFA1
:1016200001200149087010BD1002002008020020AE
:10163000001802400C02002072B600BFFEE7000056
:1016400010B504F0BBFB04465E480078844209D024
:1016500000205D4908605D49086001205C49087010
:1016600058480470002C53D15A48007830B10020FB
:10167000FFF71EFE0020584908601FE0524800682E
:1016800056490968884206D20120FFF711FE012061
:101690005149086012E051480068514909680844FE
:1016A00049490968884206D90020FFF701FE002059
:1016B0004949086002E00020434908604948007831
:1016C00018B10020FFF77CFD7AE0404800684649E9
:1016D0000968884203D20120FFF772FD70E042489A
:1016E000006842490968084438490968884203D9B2
:1016F0000020FFF765FD63E00020344908603C48A6
:10170000007808B9012000E000203949087057E04E
:101710000020FFF7CDFD00202F49086031480078F8
:1017200018B10020FFF74CFD4AE02948007828B3A3
:10173000264800682F490968884203D20120FFF734
:101740003FFD3DE02B4800682B49096808441F49CC
:101750000968884203D90020FFF732FD30E00020FD
:101760001A4908602248007808B9012000E00020EA
:101770001F49087000201649087021E013480068CE
:101780001E490968884203D20120FFF719FD17E0BE
:101790001A4800681A49096808440C4909688842CF
:1017A00003D90020FFF70CFD0AE00020074908607C
:1017B0000F48007808B9012000E000200C490870AB
:1017C00010BD0000320100201C010020200100207B
:1017D00025010020440000202C010020B40000203E
:1017E000B800002045000020BC000020C000002000
:1017F00024010020CC000020D0000020C4000020E4
:10180000C800002038B580210D48FEF713FD0020E8
:101810000C4908800CA003F0A1F80EA10848FEF7BF
:1018200014FD04465CB16A460CA12046FEF748FD53
:10183000012803D1009840B20B49087000BF38BDA1
:10184000100500204C00002041542B4353510D0A39
:10185000000000002B4353513A0000002B4353512A
:101860003A202564000000005100002030B50246F7
:10187000854C8869A04200D000BF00BF92F83C00B0
:10188000012801D1022030BD012082F83C0000BFB8
:101890000868092816D91068C0680C780A3C04EB5F
:1018A00044050724AC40A0431468E0600C780A3C6F
:1018B00004EB44048868A0401468E468204314687A
:1018C000E06013E0106800690C7804EB440507241D
:1018D000AC40A043146820610C7804EB4404886891
:1018E000A040146824692043146820611068806B4C
:1018F00020F440101468A0631068846B088A401EAE
:1019000044EA00501468A0630879C01C0C7C001BDA
:1019100000EB80041F20A0401468A46B844310686F
:1019200084630879C01C0C7C001B00EB80040888D1
:1019300080B2A0401468A46B20431468A063524C8A
:101940008869A04218D01068806820F4702014685C
:10195000A060106880688C6920431468A0601068DB
:10196000806820F440101468A06010688068CC691A
:1019700020431468A0600BE01068806820F4702099
:101980001468A0601068806820F440101468A0609B
:10199000487D30B11068406840F480601468606031
:1019A00005E01068406820F4806014686060087D7D
:1019B00030B11068406840F480501468606005E001
:1019C0001068406820F480501468606048680128FE
:1019D00004D002280FD0032827D119E010684069ED
:1019E0006FF30B001468606110684069CC68204395
:1019F0001468606126E0106880696FF30B0014685A
:101A0000A06110688069CC6820431468A06119E067
:101A10001068C0696FF30B001468E0611068C0695A
:101A2000CC6820431468E0610CE01068006A6FF332
:101A30000B00146820621068006ACC6820431468A8
:101A4000206200BF00BF114B114C1068A04206D1AC
:101A50000868122803D1586840F4800058600C4C84
:101A60001068A04209D10868102802D0086811281F
:101A700003D1586840F40000586000BF002082F88D
:101A80003C0000BF00BFFEE601000F000023014044
:101A90000020014038B502460020009000BF92F8B7
:101AA0003C00012801D1022038BD012082F83C0011
:101AB00000BF0868092816D91068C0680C780A3C6D
:101AC00004EB44050724AC40A0431468E0600C78A4
:101AD0000A3C04EB44048868A0401468E46820438E
:101AE0001468E06013E0106800690C7804EB4405AA
:101AF0000724AC40A043146820610C7804EB440434
:101B00008868A040146824692043146820614868EC
:101B1000072817D21068406B0C79641E04EB84050B
:101B20001F24AC40A04314686063088880B20C791D
:101B3000641E04EB8404A0401468646B20431468A2
:101B4000606331E048680D2817D21068006B0C798B
:101B5000E41F04EB84051F24AC40A04314682063F9
:101B6000088880B20C79E41F04EB8404A040146858
:101B7000246B20431468206316E01068C06A0C7957
:101B80000D3C04EB84051F24AC40A0431468E062C4
:101B9000088880B20C790D3C04EB8404A0401468E2
:101BA000E46A20431468E062194B1A4C1068A042A2
:101BB00006D10868122803D1586840F480005860A4
:101BC000144C1068A0421CD10868102802D0086884
:101BD000112816D1586840F4000058600868102891
:101BE0000FD10D4800680D4CB0FBF4F000EB800005
:101BF0004000009002E00098401E009000980028ED
:101C0000F9D100BF002082F83C0000BF00BF4BE7C5
:101C100000230140002001403400002040420F001A
:101C200001460868C06C704770B5044600250CB9C1
:101C3000012070BD1549A06A884200D000BF206C09
:101C400030B9204600F024F80020606484F83C009D
:101C5000206C00F0100088B9206C20F4885040F00F
:101C6000020020642046FFF70DF900206064206C1C
:101C700020F0020040F00100206400E0012500BFD8
:101C8000002084F83C0000BF2846D2E70100000F86
:101C900010B586B00446142101A8FEF7CBFA194905
:101CA000206888422CD100BF0020009016480068B0
:101CB00040F48060144908600846006800F48060C1
:101CC000009000BF00BF00BF002000900E481438F5
:101CD000006840F020000C4914390860084600688C
:101CE00000F02000009000BF00BF4FF4AC700190E6
:101CF000032002900020039001A9044800F04EFB4D
:101D000006B010BD002201404438024000140240D9
:101D100070B504460D4600262068806800F4806097
:101D2000B0F5806F11D12068806800F48070B0F544
:101D3000807F0AD1206C40F02000206400BF00208A
:101D400084F83C0000BF012070BD00F02FFC064667
:101D500018E0681CB0B125B100F028FC801BA84237
:101D600010D92068006800F0020002280AD0206C18
:101D700040F00400206400BF002084F83C0000BF55
:101D80000320E1E72068006800F002000228E0D1AB
:101D90006FF0120021680860206C40F4007020642D
:101DA0002068806800F04050B8B9207EA8B920684B
:101DB000C06A00F4700020B12068806800F4806080
:101DC00058B9206C20F480702064206C00F480509E
:101DD00018B9206C40F0010020640020B4E7000036
:101DE00008B501460020009000BF91F83C00012892
:101DF00001D1022008BD012081F83C0000BF086825
:101E0000806800F00100A0B90868806840F0010017
:101E10000B6898603F4800683F4BB0FBF3F000EB65
:101E20004000009002E00098401E009000980028BA
:101E3000F9D10868806800F00100002860D0086CC3
:101E400040F20163984340F4807008640868406879
:101E500000F4806028B1086C20F4005040F48050F9
:101E60000864086C00F48050B0F5805F04D1486CC1
:101E700020F00600486401E00020486400BF002014
:101E800081F83C0000BF254A6FF022000B68186003
:101E9000506800F01F0018BB214B0868984213D00F
:101EA000204B0868984204D1101D006800F01F0004
:101EB00050B11D4B086898422AD11848001D00688F
:101EC00000F01F00102823D20868806800F04050FE
:101ED000F0B90868806840F080400B68986017E0AF
:101EE0000F4B0868984213D10868806800F0405092
:101EF00070B90868806840F080400B68986007E01F
:101F0000086C40F010000864486C40F00100486420
:101F100000206FE73400002040420F000023014002
:101F2000002001400021014000220140014600BF85
:101F300091F83C00012801D102207047012081F86E
:101F40003C0000BF0868806820F001000A689060CB
:101F50000868806800F0010028B9086C20F48850F7
:101F600040F00100086400BF002081F83C0000BF81
:101F700000BFE2E770B50446A56D00F017FB06460A
:101F800094F83500022808D08020606500BF00204A
:101F900084F8340000BF012070BD2068006820F084
:101FA0001600216808602068406920F080002168E0
:101FB0004861206C08B9A06C28B12068006820F046
:101FC0000800216808602068006820F0010021688E
:101FD000086010E000F0EAFA801B05280BD92020E9
:101FE0006065032084F8350000BF002084F83400C9
:101FF00000BF0320D0E72068006800F0010000283F
:10200000E8D194F85C103F208840A860012084F853
:10201000350000BF002084F8340000BF00BFBBE7DC
:10202000014691F83500022803D080204865012040
:102030007047052081F835000868006820F001002D
:102040000A6810600020F3E7F8B50446002000900D
:102050008C4800684FF41651B0FBF1F7A56D2E685F
:1020600094F85C1008208840304098B120680068DF
:1020700000F0040070B12068006820F004002168BE
:10208000086094F85C1008208840A860606D40F0FB
:102090000100606594F85C1001208840304068B110
:1020A0002068406900F0800040B194F85C10012085
:1020B0008840A860606D40F00200606594F85C1094
:1020C00004208840304068B12068006800F00200B9
:1020D00040B194F85C1004208840A860606D40F026
:1020E0000400606594F85C1010208840304078B39C
:1020F0002068006800F0080050B394F85C101020CD
:102100008840A8602068006800F4802080B12068C2
:10211000006800F4002028B9206CC8B12046216C6A
:10212000884715E0A06C98B12046A16C88470FE065
:102130002068006800F4807028B92068006820F0EA
:10214000080021680860206C10B12046216C884787
:1021500094F85C10202088403040002865D020682A
:10216000006800F0100000285FD094F85C10202078
:102170008840A86094F83500052828D120680068B8
:1021800020F01600216808602068406920F0800077
:1021900021684861206C08B9A06C28B120680068EB
:1021A00020F008002168086094F85C103F20884007
:1021B000A860012084F8350000BF002084F83400B6
:1021C00000BF206D10B12046216D8847F8BD206802
:1021D000006800F4802080B12068006800F40020CE
:1021E00028B9606C10B12046616C88471DE0E06B37
:1021F000D8B12046E16B884717E02068006800F4FA
:10220000807068B92068006820F0100021680860BC
:10221000012084F8350000BF002084F8340000BF9E
:10222000E06B10B12046E16B8847606D38B3606D9C
:1022300000F00100F0B1052084F835002068006846
:1022400020F001002168086000BF0098401C009049
:10225000B84200D905E02068006800F001000028BD
:10226000F3D100BF012084F8350000BF002084F8BE
:10227000340000BFE06C10B12046E16C884700BF1D
:10228000A4E70000340000202DE9F04104460025B9
:1022900000F08CF9074614B90120BDE8F081606AAE
:1022A00000B100BF022084F8350000BF002084F890
:1022B000340000BF2068006820F001002168086039
:1022C0000AE000F073F9C01B052805D920206065DD
:1022D000032084F83500E0E72068006800F0010082
:1022E0000028EED12068056821480540D4E90101A5
:1022F0000843E16808432169084361690843A1690B
:102300000843E1690843216A08430543606A0428D9
:1023100003D1D4E90B010843054320680560206818
:10232000456925F00705606A0543606A04280DD1F8
:10233000A06A0543E06A48B12046FEF7EDFF28B1E8
:1023400040206065012084F83500A6E720684561DB
:102350002046FEF7C7FF064694F85C103F208840F1
:10236000B06000206065012084F83500002094E70B
:102370003F8010F070B5044600F018F90646254677
:10238000681C10B104480078054400BF00F00EF945
:10239000801BA842FAD370BD30000020F8B5024679
:1023A0000B460025002400200021D6E0012606FA75
:1023B00001F51E6806EA0504AC4274D11E7906F0E8
:1023C0000306012E04D01E7906F00306022E13D157
:1023D00090684F000326BE40B0434F00DE68BE4009
:1023E00030439060506801268E40B0431E79C6F39A
:1023F00000168E40304350601E7906F00306032E0F
:1024000009D0D0684F000326BE40B0434F009E68FD
:10241000BE403043D0601E7906F00306022E13D171
:10242000CF0802F1200656F827004E07F70E0F26B8
:10243000BE40B0434F07FF0E1E69BE403043CF0879
:1024400002F1200646F8270010684F000326BE4020
:10245000B0431E7906F003064F00BE4030431060C3
:102460005E6806F44036002E76D000BF0026009647
:102470003C4E366846F480463A4F3E603E463668EB
:1024800006F48046009600BF00BF374E8F0856F80E
:1024900027008E07370F0F26BE40B043334EB2429F
:1024A00002D1002624E057E0314EB24201D101268C
:1024B0001EE0304EB24201D1022619E02E4EB24249
:1024C00001D1032614E02D4EB24201D104260FE0C3
:1024D0002B4EB24201D105260AE02A4EB24201D16A
:1024E000062605E0284EB24201D1072600E0082664
:1024F0008F073F0FBE4030431B4E8F0846F8270022
:10250000224E3068A0435E6806F4801606B1204370
:102510001E4E3060361D3068A0435E6806F400161B
:1025200006B12043194E361D3060184E361F3068F4
:10253000A0435E6806F4003606B12043134E361FF2
:102540003060361F3068A0435E6806F4803606B1FE
:1025500020430E4E083E3060491C1029FFF426AF80
:10256000F8BD000044380240083801400000024035
:102570000004024000080240000C0240001002402B
:102580000014024000180240001C0240083C0140B8
:10259000024613690B400BB1012000E00020704798
:1025A0000AB1816101E00B04836170470148006852
:1025B000704700002800002070B504460CB90120C7
:1025C00070BD94F83D0028B9002084F83C002046F6
:1025D00000F010FB242084F83D002068006820F003
:1025E0000100216808602068006840F4004021680C
:1025F00008602068006820F400402168086000F04E
:10260000DFFC05465C496068884206D85B48854225
:1026100001D2012007E0002005E05948854201D29F
:10262000012000E00020012800D1C9E75548B5FB92
:10263000F0F62068406820F03F0030432168486091
:102640004D496068884201D8701C07E04FF49670CD
:1026500070434FF47A71B0FBF1F0401C2168096AB5
:1026600021F03F01084321680862434960688842BD
:1026700014D8681E61684900B0FBF1F0401CC0F33B
:102680000B00042801D204203DE0681E6168490067
:10269000B0FBF1F0401CC0F30B0034E0A06838B987
:1026A000681E616801EB4101B0FBF1F0401C0AE0DB
:1026B000681E616801EBC10202EB0111B0FBF1F091
:1026C000401C40F48040C0F30B0008B901201AE020
:1026D000A06848B9681E616801EB4101B0FBF1F0E8
:1026E000401CC0F30B000CE0681E616801EBC102E6
:1026F00002EB0111B0FBF1F0401CC0F30B0040F401
:10270000804040F400402168C9694CF6FF72914353
:1027100008432168C861D4E90701084321680968B2
:1027200021F0C001084321680860D4E90310084380
:102730002168896848F2FF32914308432168886024
:10274000D4E9050108432168C96821F0FF01084365
:102750002168C8602068006840F0010021680860B6
:1027600000202064202084F83D000020206384F8AD
:102770003E0000BF24E70000A086010080841E0008
:1027800000093D0040420F002DE9FC5F04460F4662
:1027900090469946DDE90CAB0E9EFFF707FF054614
:1027A00094F83D00202870D119230122B549204614
:1027B000009501F05AFF10B10220BDE8FC9F00BF58
:1027C00094F83C00012801D10220F6E7012084F8AA
:1027D0003C0000BF2068006800F0010028B92068B4
:1027E000006840F00100216808602068006820F45B
:1027F000006021680860222084F83D00402084F8B1
:102800003E0000202064C4F824A0A4F82AB0608D03
:1028100020859D48E0624B46424639462046CDE938
:10282000006501F0CFFD08B10120C6E7208D88B911
:1028300000BF0020019020684069019020688069F5
:10284000019000BF00BF2068006840F4007021685C
:10285000086040E0208D012818D12068006820F42D
:1028600080602168086000BF0020019020684069F6
:10287000019020688069019000BF00BF2068006857
:1028800040F400702168086025E0F8E0208D0228FF
:1028900016D12068006820F48060216808602068F4
:1028A000006840F400602168086000BF00200190CB
:1028B00020684069019020688069019000BF0AE0AB
:1028C00000BF002001902068406901902068806965
:1028D000019000BF00BFC3E0208D03287ED8208D6B
:1028E000012815D12A463146204601F09AFF08B149
:1028F000012062E720680069616A0870606A401C14
:102900006062208D401E2085608D401E6085A7E09E
:10291000208D02282AD1334600225C4920460095AA
:1029200001F0A3FE08B1012047E72068006840F4E9
:1029300000702168086020680069616A0870606A38
:10294000401C6062208D401E2085608D401E608589
:1029500020680069616A0870606A401C6062208DAE
:10296000401E2085608D401E608579E03346002240
:1029700046492046009501F078FE08B101201CE789
:102980002068006820F48060216808602068006981
:10299000616A0870606A401C6062208D401E20855C
:1029A000608D401E608533460022384920460095E0
:1029B00001F05BFE08B10120FFE62068006840F4EA
:1029C00000702168086020680069616A0870606AA8
:1029D000401C6062208D401E208500E010E0608D6C
:1029E000401E608520680069616A0870606A401C4A
:1029F0006062208D401E2085608D401E60852FE026
:102A00002A463146204601F00CFF08B10120D4E6E9
:102A100020680069616A0870606A401C6062208DED
:102A2000401E2085608D401E608520684069C0F38F
:102A30008000A8B1208D032805D12068006820F40B
:102A400080602168086020680069616A0870606AB7
:102A5000401C6062208D401E2085608D401E608578
:102A6000208D00287FF438AF202084F83D0000201E
:102A700084F83E0000BF84F83C0000BF9DE60220C1
:102A80009BE60000020010000000FFFF04000100B0
:102A90002DE9FC5F04460F4690469946DDE90CABF4
:102AA0000E9EFFF783FD054694F83D0020287DD15A
:102AB000192301224D492046009501F0D6FD10B1A1
:102AC0000220BDE8FC9F00BF94F83C00012801D122
:102AD0000220F6E7012084F83C0000BF206800686F
:102AE00000F0010028B92068006840F0010021686A
:102AF00008602068006820F40060216808602120D8
:102B000084F83D00402084F83E0000202064C4F892
:102B100024A0A4F82AB0608D20853548E0624B4699
:102B2000424639462046CDE9006501F0FBFC08B17C
:102B30000120C6E731E02A463146204601F0B6FEC4
:102B400050B1206C042805D12068006840F4007062
:102B5000216808600120B4E7606A00782168086194
:102B6000606A401C6062208D401E2085608D401E82
:102B7000608520684069C0F3800070B1208D60B12D
:102B8000606A007821680861606A401C6062208D7C
:102B9000401E2085608D401E6085208D0028CAD192
:102BA0002A463146204601F02DFD00E01CE050B1E0
:102BB000206C042805D12068006840F4007021686A
:102BC000086001207DE72068006840F400702168FB
:102BD0000860202084F83D00002084F83E0000BFFB
:102BE00084F83C0000BF6CE702206AE70200100096
:102BF0000000FFFF10B586B00446142101A8FDF7C0
:102C000019FB1B49206888422FD100BF002000908B
:102C10001848006840F0200016490860084600681F
:102C200000F02000009000BF00BF032001901220A0
:102C3000029000200390032004900420059001A935
:102C40000D48FFF7ABFB00BF002000900948103093
:102C5000006840F4800007491031086008460068A9
:102C600000F48000009000BF00BF06B010BD00005F
:102C70000058004030380240001402400348006809
:102C8000034909780844014908607047280000207A
:102C90003000002010B50D48006840F400700B496A
:102CA00008600846006840F48060086008460068D4
:102CB00040F480700860032000F0A6F80F2000F0B8
:102CC00007F800F02BF8002010BD0000003C024087
:102CD00070B504460E4800784FF47A71B1FBF0F0FD
:102CE0000C490968B1FBF0F5284600F02FFC08B14B
:102CF000012070BD102C07D200222146501E00F08A
:102D000045F80548046001E00120F2E70020F0E703
:102D100030000020340000202C00002008B500BF47
:102D2000002000900E48006840F480400C49086084
:102D30000846006800F48040009000BF00BF00BF5C
:102D400000200090081F006840F08050091F0860B4
:102D50000846006800F08050009000BF00BF08BD2A
:102D6000443802400146084600280DDB00BF00BF82
:102D700000F01F0301229A4043099B0003F1E02366
:102D8000C3F8002100BF00BF00BF70472DE9F05F0E
:102D900080460D461646002704F0B0F9074639462E
:102DA0002A46334601F00700C0F1070ABAF1040FC2
:102DB00002D94FF0040A01E0C0F1070AD14600F140
:102DC000040ABAF1070F02D24FF0000A01E0A0F1A5
:102DD000030AD4464FF0010A0AFA09FAAAF1010AD5
:102DE0000AEA020A0AFA0CFA4FF0010B0BFA0CFB82
:102DF000ABF1010B0BEA030B4AEA0B0421464046F8
:102E000004F084F9BDE8F09F00BF00F00702064B14
:102E100019684FF6FF031940044B0B4343EA0221A4
:102E2000014B196000BF70470CED00E00000FA058F
:102E300070B504460D460CB9012070BD58480068B5
:102E400000F00700A84209D255490D7008460068F5
:102E500000F00700A84201D00120EEE7207800F042
:102E6000020002281DD1207800F00400042805D1BA
:102E70004C48006840F4E0504A490860207800F06F
:102E80000800082805D14748006840F460404549DB
:102E900008604448006820F0F000A16808434149F8
:102EA0000860207800F00100A8B36068012807D10D
:102EB0003C4808380068C0F34040B8B90120BCE77E
:102EC0006068022802D06068032807D135480838B6
:102ED0000068C0F3406048B90120AEE731480838C7
:102EE0000068C0F3400008B90120A6E72D4800683B
:102EF00020F00300616808432A490860FFF756FB89
:102F0000064609E0FFF752FB801B41F288318842F8
:102F100002D9032091E707E02248006800F00C0086
:102F20006168B0EB810FEDD11D48006800F007002B
:102F3000A84209D91A490D700846006800F0070038
:102F4000A84201D0012078E7207800F0040004288E
:102F500007D11448006820F4E050E16808431149A3
:102F60000860207800F00800082808D10D480068A3
:102F700020F46040216940EAC1000A49086000F07D
:102F80003FF808490968C1F30311074A515CC8407A
:102F90000649086006480068FFF79AFE00204CE7E3
:102FA000003C024008380240DC8000083400002069
:102FB0002C00002001480068704700003400002009
:102FC00000B5FFF7F7FF04490968C1F38221034AFE
:102FD000515CC84000BD000008380240EC80000889
:102FE00000B5FFF7E7FF04490968C1F34231034A1E
:102FF000515CC84000BD000008380240EC80000869
:103000002DE9F047002400250026A1462548006848
:1030100000F00C0020B1042805D008283AD105E0C2
:10302000DFF8849039E0DFF8849036E01D48001F17
:10303000006800F03F041B48001F006800F4800097
:1030400078B11A481749091F0968C1F38811A0FB14
:1030500001700146224600233846FDF7B3F80546C5
:103060000EE011480F49091F0968C1F38811A0FB40
:1030700001700146224600233846FDF7A3F80546B5
:103080000848001F0068C0F30140401C4600B5FB23
:10309000F6F902E0DFF8109000BF00BF4846BDE837
:1030A000F0870000083802400024F40000127A0083
:1030B000F8B504460CB90120F8BD207800F00100F5
:1030C000002874D0F948006800F00C0004280DD0E6
:1030D000F648006800F00C00082813D1F348001FE0
:1030E000006800F48000B0F5800F0BD1EF4808387D
:1030F0000068C0F34040002859D06068002856D1CD
:103100000120D9E700BF6068B0F5803F08D1E748EB
:103110000838006840F48030E449083908601EE04F
:103120006068B0F5A02F0DD1E0480838006840F481
:103130008020DE49083908600846006840F4803085
:1031400008600CE0D9480838006820F48030D7497E
:10315000083908600846006820F48020086000BF35
:10316000606890B1FFF722FA054606E0FFF71EFA05
:10317000401B642801D903209EE7CC48083800682A
:10318000C0F340400028F1D011E0FFF70FFA0546E8
:1031900006E0FFF70BFA401B642801D903208BE7F8
:1031A000C24808380068C0F340400028F1D12078B8
:1031B00000F0020002285FD1BC48006800F00C005B
:1031C00058B1BA48006800F00C0008281CD1B74874
:1031D000001F006800F48000B0B9B44808380068E7
:1031E000C0F3400020B1E068012801D0012063E76E
:1031F000AE480838006820F0F800216940EAC100B4
:10320000AA490839086037E0E06800B30120A849FE
:103210000860FFF7CBF9054606E0FFF7C7F9401B4A
:10322000022801D9032047E7A04808380068C0F306
:1032300040000028F1D09D480838006820F0F800D0
:10324000216940EAC10099490839086014E000206A
:1032500097490860FFF7AAF9054606E0FFF7A6F9C7
:10326000401B022801D9032026E79048083800684F
:10327000C0F340000028F1D1207800F008000828B1
:103280002CD16069A8B101208A490860FFF78EF946
:10329000054606E0FFF78AF9401B022801D9032002
:1032A0000AE782486C300068C0F340000028F1D083
:1032B00014E000207F490860FFF778F9054606E032
:1032C000FFF774F9401B022801D90320F4E6774880
:1032D0006C300068C0F340000028F1D1207800F085
:1032E0000400042870D1002770483830006800F0CE
:1032F000805090B900BF002000906C4838300068C2
:1033000040F080506949383108600846006800F094
:103310008050009000BF00BF01276748006800F49C
:103320008070B0B96448006840F4807062490860F9
:10333000FFF73CF9054606E0FFF738F9401B022885
:1033400001D90320B8E65C48006800F480700028CA
:10335000F2D000BFA068012808D154486830006846
:1033600040F001005149683108601DE0A06805285F
:103370000DD14E486830006840F004004B49683178
:1033800008600846006840F0010008600CE047480B
:103390006830006820F00100444968310860084640
:1033A000006820F00400086000BFA068A8B1FFF723
:1033B000FDF8054609E0FFF7F9F8401B41F28831B6
:1033C000884202D9032077E626E038486830006852
:1033D000C0F340000028EED013E0FFF7E7F8054601
:1033E00008E0FFF7E3F8401B41F28831884201D939
:1033F000032061E62D4868300068C0F340000028D3
:10340000EFD1012F07D129483830006820F08050D3
:1034100026493831086000BFA069002845D02348FC
:10342000006800F00C0008285DD0A069022845D192
:1034300000201F490866FFF7B9F8054606E0FFF7C8
:10344000B5F8401B022801D9032035E61748083893
:103450000068C0F340600028F1D1D4E907010843B7
:10346000616A40EA81110122A06AC2EB500041EA80
:1034700000412C20005D41EA00600C49091F0860F2
:1034800001200B490866FFF791F8054606E0FFF7B3
:103490008DF8401B022801D903200DE603480838A7
:1034A0000068C0F340600028F1D049E008380240CD
:1034B00000004742800E4742007000400020214932
:1034C0000866FFF773F8054606E0FFF76FF8401B44
:1034D000022801D90320EFE51B480068C0F34060D3
:1034E0000028F2D12CE0A069012800D1E4E51648BB
:1034F000001D0668A069012820D006F48001E0695B
:1035000081421BD106F03F01206A814216D147F665
:10351000C0703040616AB0EB811F0FD106F44031BA
:103520000122A06AC2EB5000B1EB004F06D106F0B9
:1035300070612C20005DB1EB006F01D00120BBE574
:103540000020B9E5000047420038024070B504464B
:103550002546681EB0F1807F01D301200FE0681E70
:103560004FF0E02148610F214FF0FF3003F0CEFD16
:1035700000204FF0E021886107200861002070BD25
:103580007047704730B502460B4600BF92F83C00CA
:10359000012801D1022030BD012082F83C0000BF8B
:1035A000022082F83D00106844681068816824F0A9
:1035B00070041868044310684460184D1068A842ED
:1035C0001BD01068B0F1804F17D0154D1068A8427D
:1035D00013D0144D1068A8420FD0134D1068A842A4
:1035E0000BD0124D1068A84207D0114D1068A842A8
:1035F00003D0104D1068A84205D121F08001586811
:10360000014310688160012082F83D0000BF002066
:1036100082F83C0000BF00BFBDE700000000014091
:103620000004004000080040000C0040000401407D
:10363000004001400018004010B504460CB90120BC
:1036400010BD94F83D0028B9002084F83C002046C5
:1036500000F026F8022084F83D00211D206802F0C9
:10366000E9FE012084F8460000BF84F83E000121F5
:103670003F200155402001554120015500BF00BFAA
:10368000012084F842004320015544200155452083
:10369000015500BF012084F83D000020D0E7000064
:1036A00038B504462068B0F1804F18D100BF002023
:1036B00000903648006840F0010034490860084630
:1036C000006800F00100009000BF00BF002203214D
:1036D0001C20FFF75BFB1C20FFF744FB55E02C4947
:1036E0002068884218D100BF002000902748006859
:1036F00040F00200254908600846006800F002001A
:10370000009000BF00BF002211461D20FFF73EFBC6
:103710001D20FFF727FB38E01E492068884218D19A
:1037200000BF002000901948006840F010001749C1
:1037300008600846006800F01000009000BF00BF5D
:10374000002211463620FFF721FB3620FFF70AFB47
:103750001BE011492068884217D100BF002000906B
:103760000A48006840F020000849086008460068E0
:1037700000F02000009000BF00BF0022114637205B
:10378000FFF704FB3720FFF7EDFA38BD4038024061
:10379000000400400010004000140040014691F871
:1037A0003D00012801D001207047022081F83D0032
:1037B0000868C06840F001000B68D8601A4B0868C0
:1037C00098421BD00868B0F1804F17D0174B08689B
:1037D000984213D0164B086898420FD0154B0868D2
:1037E00098420BD0144B0868984207D0134B0868D6
:1037F000984203D0124B086898420CD10868806840
:1038000000F00702062A0CD00868006840F00100AA
:103810000B68186005E00868006840F001000B685C
:1038200018600020C0E700000000014000040040D4
:1038300000080040000C004000040140004001402E
:103840000018004001460868C06820F001000A68BE
:10385000D06000BF0868006A41F21112104050B9F0
:103860000868006A9210104028B90868006820F0C3
:1038700001000A68106000BF012081F83D000020AF
:1038800070472DE9F04104460D46002700BF94F82B
:103890003C00012802D10220BDE8F081012084F81B
:1038A0003C0000BF022084F83D002068866826F0B6
:1038B000770626F47F46206886602868502833D033
:1038C0000CDC202850D004DC00284BD0102851D12B
:1038D00049E0302849D040284CD139E060282DD02B
:1038E000702807D0B0F5805F03D0B0F5005F41D1FC
:1038F0000DE041E0D5E902136A68206802F00EFE8F
:103900002068866846F077062068866034E0D5E94E
:1039100002136A68206802F001FE2068806840F4A3
:1039200080402168886027E0EA686968206802F0C2
:1039300009FE5021206802F0FCFD1DE0EA6869687C
:10394000206802F012FE6021206802F0F2FD13E010
:10395000EA686968206802F0F5FD4021206802F0FD
:10396000E8FD09E000BF00BF00BF2968206802F041
:10397000E0FD01E0012700BF00BF012084F83D0009
:1039800000BF002084F83C0000BF384684E7704741
:1039900070B504462068C5682068066906F0020014
:1039A000022819D105F00200022815D1401F216814
:1039B0000861012020772068806900F0030018B1B9
:1039C0002046FFF7E4FF05E0204600F097F8204688
:1039D00000F095F80020207706F00400042819D1A3
:1039E00005F00400042815D1C043216808610220B5
:1039F00020772068806900F4407018B12046FFF7F6
:103A0000C6FF05E0204600F079F8204600F077F880
:103A10000020207706F00800082819D105F00800DA
:103A2000082815D1C0432168086104202077206848
:103A3000C06900F0030018B12046FFF7A8FF05E0B9
:103A4000204600F05BF8204600F059F8002020776F
:103A500006F01000102819D105F01000102815D11B
:103A6000C04321680861082020772068C06900F4FD
:103A7000407018B12046FFF78AFF05E0204600F0AD
:103A80003DF8204600F03BF80020207706F00100CA
:103A900048B105F0010030B16FF001002168086104
:103AA000204600F02DF806F08000802809D105F0AE
:103AB0008000802805D1C043216808612046FFF7B7
:103AC0005FFD06F04000402809D105F04000402885
:103AD00005D1C04321680861204600F0A9F806F02E
:103AE0002000202809D105F02000202805D1C0435E
:103AF000216808612046FFF744FD70BD704770479C
:103B000010B5044637492068884211D136480088EC
:103B1000401C354908800846008841F288318842B7
:103B20005EDB00203049088001203049087057E0F2
:103B30002068B0F1804F34D12D48007898B12D48DD
:103B40000068401C2B490860084600683C2809D3DF
:103B5000002029490860264908702649086027A0E6
:103B600003F0A8FA10BD29480078B8B922480068C7
:103B7000401C2149086026480068401C2449086010
:103B800024480078042809D123480068401C2249B1
:103B9000086022480068401C2049086001F0B2FF1C
:103BA0001EE01F492068884219D11E480068401C49
:103BB0001C4908603C2813D3002008601A4800689C
:103BC000401C194908603C2806D3002008601748AB
:103BD0000068401C15490860FDF704FD00E000BFC7
:103BE00000BFBFE700100040100000205000002080
:103BF0002A010020140000201C0100203F3F3F3F0D
:103C00003F3F3F3F3F3F3F3F3F3F0A0029010020EA
:103C100020010020180100201001002014010020C4
:103C20000014004004020020080200200C020020C2
:103C30007047F8B504460E46174694F8420020280F
:103C40002ED106B10FB90120F8BD0120206300205C
:103C500060633A463146204602F0DCFF0546EDB986
:103C6000206B012819D100BF002000902068006857
:103C7000009020684068009000BF00BF00BF00BFF8
:103C800021680C3151E8001F41F0100021680C310F
:103C900041E80002002AF3D100E001252846D3E7DD
:103CA0000220D1E770B505460C46064928688842CF
:103CB00006D105480480802204490548FFF7B9FF72
:103CC00070BD0000004400404C00002010050020A2
:103CD00068040020704700002DE9F84F0446206872
:103CE00005682068C668206847694FF00009CA4621
:103CF00005F00F09B9F1000F0AD105F0200038B125
:103D000006F0200020B1204602F0F0FDBDE8F88F5B
:103D1000B9F1000F7CD007F0010018B906F49070DB
:103D2000002875D005F0010030B106F4807018B19C
:103D3000606C40F00100606405F0040030B107F0F1
:103D4000010018B1606C40F00200606405F00200F0
:103D500030B107F0010018B1606C40F004006064FD
:103D600005F0080048B106F0200010B907F0010086
:103D700018B1606C40F008006064606C002846D0A8
:103D800005F0200028B106F0200010B1204602F016
:103D9000ADFD20684069C0F3801A606C00F0080037
:103DA00010B9BAF1000F2DD0204602F059FD20685D
:103DB000406900F04000402820D100BF00BF2168CA
:103DC000143151E8001F21F040002168143141E80E
:103DD0000002002AF3D100BFE06B50B17748E16BDD
:103DE0000865E06BFEF71CF988B1E06B016D884750
:103DF0000DE02046FFF76EFF09E009E02046FFF7DF
:103E000069FF04E02046FFF765FF002060647DE75E
:103E1000206B012878D105F01000002874D006F03E
:103E200010000028FAD000BF002000902068006831
:103E3000009020684068009000BF00BF2068406983
:103E400000F04000402860D1E06B006840681FFA35
:103E500080F8B8F1000F56D0A08D404553DDA4F88E
:103E60002E80E06BC069B0F5807F43D000BF00BFFB
:103E700021680C3151E8001F21F4807021680C3159
:103E800041E80002002AF3D100BF00BF00BF216853
:103E9000143151E8001F21F001002168143141E87C
:103EA0000002002AF3D100BF00BF00BF2168143117
:103EB00051E8001F21F040002168143141E8000260
:103EC000002AF3D100BF202084F8420000202063A4
:103ED00000BF00BF21680C3151E8001F21F0100025
:103EE00021680C3141E80002002AF3D100BFE06BE9
:103EF000FEF740F802206063A08DE28D801A81B247
:103F00002046FFF7CFFE01E742E0A08DE18D401A89
:103F10001FFA80F8E08DD0B3B8F1000F37D000BFA2
:103F200000BF21680C3151E8001F21F49070216816
:103F30000C3141E80002002AF3D100BF00BF00BFEE
:103F40002168143151E8001F21F00100216814316B
:103F500041E80002002AF3D100BF202084F842008B
:103F60000020206300BF00BF21680C3151E8001F12
:103F700021F0100021680C3141E80002002AF3D141
:103F800000BF0220606341462046FFF78BFEBDE67E
:103F900005F0800030B106F0800018B1204602F034
:103FA00059FEB3E605F0400030B106F0400018B10C
:103FB000204602F08BFCA9E600BFA7E64D6800088A
:103FC00010B504460CB9012010BDA06900B100E095
:103FD00000BF94F8410028B9002084F84000204632
:103FE00000F02AF8242084F841002068C06820F4FA
:103FF00000502168C860204602F0F6FC2068006985
:1040000020F49040216808612068406920F02A006F
:10401000216848612068C06840F400502168C86089
:1040200000206064202084F8410084F842000020D1
:10403000606300BFC8E7000010B586B004461421D5
:1040400001A8FCF7F7F869492068884257D100BFFA
:10405000002000906648006840F400206449086031
:104060000846006800F40020009000BF00BF00BFB9
:10407000002000905E481038006840F001005C4964
:10408000103908600846006800F00100009000BF89
:1040900000BF032001900220029000200390032023
:1040A00004900820059001A95248FEF777F952487C
:1040B0005249086040054860002150488160C16055
:1040C0004FF4806101610021416181614FF4807191
:1040D000C161002101624162FEF7D6F808B1FDF727
:1040E000ABFA00BF4548E063846300BF002211467D
:1040F0003420FEF74BFE3420FEF734FE73E04049D7
:104100002068884233D100BF002000903848001D4D
:10411000006840F010003649091D08600846006834
:1041200000F01000009000BF00BF00BF0020009012
:104130002F481038006840F001002D491039086000
:104140000846006800F00100009000BF00BF4FF477
:10415000C060019002200290002003900320049090
:104160000720059001A92348FEF718F93BE02549EF
:104170002068884237D100BF002000901C480068AA
:1041800040F400301A4908600846006800F4003026
:10419000009000BF00BF00BF0020009014481038FE
:1041A000006840F0080012491039086008460068AD
:1041B00000F00800009000BF00BF602001900220C6
:1041C000029000200390032004900720059001A98D
:1041D0000D48FEF7E3F8002202212620FEF7D6FD67
:1041E0002620FEF7BFFD06B010BD0000004C0040C9
:1041F000403802400000024040600240B00400200D
:104200000010014000440040000C024070B504461C
:104210000D46164694F8420020280BD105B10EB980
:10422000012070BD0020206332462946204602F05E
:10423000F1FCF6E70220F4E770B50446FEF7B6F9A4
:1042400005461949206888422CD118480088B0F5E5
:10425000167F1FDA16490A7814490888411C134B47
:10426000198014490A5418460088182815DB12488A
:104270000068281AB0F57A7F08D31846008840F401
:104280000040194608800C48056006E000200749F8
:10429000088002E0002005490880012204490748FF
:1042A000FFF7B4FF70BD0000004C00408401002007
:1042B0000C000020A008002024000020D8030020CB
:1042C0002DE9F84F04460E46174699464FF0000A6E
:1042D00094F84100202850D106B117B90120BDE85B
:1042E000F88F00206064212084F84100FEF75EF919
:1042F0008246A784E784A068B0F5805F04D1206976
:1043000010B90025B04602E035464FF000081EE027
:104310005346002280212046CDF8009002F0CAFCCE
:1043200020B1202084F841000320D8E745B9B8F82F
:104330000000C0F308002168486008F1020803E0AB
:104340002878216848606D1CE08C401EE084E08C79
:104350000028DDD15346002240212046CDF80090B0
:1043600002F0A8FC20B1202084F841000320B6E729
:10437000202084F841000020B1E70220AFE7704719
:1043800000BFFEE7014608684069C0F38020B0B175
:104390006FF480600A68506100200863202081F873
:1043A0003D00002081F83E00086C40F004000864E5
:1043B00000BF002081F83C0000BF012070470020B2
:1043C000FCE700002DE9F84304460F4615469946E0
:1043D000DDE908862068006840F480602168086094
:1043E0002068006840F4807021680860434600221D
:1043F0004FF001112046009600F037F960B12068B7
:10440000006800F48070B0F5807F02D14FF4007036
:1044100020640320BDE8F88307F0FE0021680861EE
:10442000334642463E49204600F07EF908B101205D
:10443000F0E700BF002000902068406900902068ED
:104440008069009000BF00BF32464146204600F020
:104450002DFA50B1206C042805D12068006840F482
:104460000070216808600120D4E7B9F1010F03D181
:10447000E8B22168086117E0C5F3072021680861E8
:1044800032464146204600F011FA50B1206C042813
:1044900005D12068006840F40070216808600120A0
:1044A000B8E7E8B22168086132464146204600F08C
:1044B000FDF950B1206C042805D12068006840F453
:1044C0000070216808600120A4E72068006840F4BB
:1044D000807021680860434600224FF00111204699
:1044E000009600F0C2F858B12068006800F48070AF
:1044F000B0F5807F02D14FF400702064032089E77B
:10450000F8B240F001002168086133464246044990
:10451000204600F009F908B101207BE7002079E787
:10452000020001002DE9F8430446884615469946E5
:10453000DDE908672068006840F480702168086041
:10454000334600224FF001112046009700F08DF80D
:1045500060B12068006800F48070B0F5807F02D1FF
:104560004FF4007020640320BDE8F88308F0FE00DB
:10457000216808613B4632462149204600F0D4F8C4
:1045800008B10120F0E700BF0020009020684069DA
:10459000009020688069009000BF00BF3A46314615
:1045A000204600F083F950B1206C042805D1206822
:1045B000006840F40070216808600120D4E7B9F178
:1045C000010F03D1E8B22168086117E0C5F30720A5
:1045D000216808613A463146204600F067F950B13B
:1045E000206C042805D12068006840F40070216820
:1045F00008600120B8E7E8B2216808610020B3E74D
:104600000200010070B504460D46164625E020461E
:10461000FFF7B8FE08B1012070BD681CE8B1FDF7D6
:10462000C5FF801BA84200D8BDB920684069C0F30F
:10463000800090B900202063202084F83D000020F5
:1046400084F83E00206C40F02000206400BF002071
:1046500084F83C0000BF0120DEE720684069C0F319
:1046600080000028D3D00020D6E72DE9F041044691
:104670000D4617461E46DDF8188038E0701CA8B3BA
:10468000FDF794FFA0EB0800B04200D876BBC5F35D
:10469000074001280AD120684069A9B20840A9B2A0
:1046A000884201D101200BE0002009E020688069E8
:1046B000A9B20840A9B2884201D1012000E000203F
:1046C000B84214D100202063202084F83D0000204F
:1046D00084F83E00206C40F02000206400BF0020E1
:1046E00084F83C0000BF0120BDE8F081FFE7C5F37E
:1046F000074001280AD120684069A9B20840A9B240
:10470000884201D101200BE0002009E02068806987
:10471000A9B20840A9B2884201D1012000E00020DE
:10472000B842ABD00020DFE72DE9F04104460D464A
:1047300016461F4658E020684069C0F38020E8B163
:104740002068006840F40070216808606FF48060A1
:104750002168486100202063202084F83D0000206B
:1047600084F83E00206C40F00400206400BF00206C
:1047700084F83C0000BF0120BDE8F081701C90B3BC
:10478000FDF714FFC01BB04200D866BBC5F307405D
:1047900001280AD120684069A9B20840A9B288421C
:1047A00001D101200BE0002009E020688069A9B256
:1047B0000840A9B2884201D1012000E0002090B950
:1047C00000202063202084F83D00002084F83E0073
:1047D000206C40F02000206400BF002084F83C00E2
:1047E00000BF0120C8E7FFE7C5F3074001280AD151
:1047F00020684069A9B20840A9B2884201D10120CD
:104800000BE0002009E020688069A9B20840A9B245
:10481000884201D1012000E0002000288BD0002038
:10482000AAE770B504460D46164637E02068406991
:10483000C0F30010A0B16FF01000216848610020A3
:104840002063202084F83D00002084F83E00206C86
:10485000206400BF002084F83C0000BF012070BD30
:10486000FDF7A4FE801BA84200D8BDB920684069AE
:10487000C0F3801090B900202063202084F83D0010
:10488000002084F83E00206C40F02000206400BF2F
:10489000002084F83C0000BF0120E0E72068406968
:1048A000C0F380100028C1D00020D8E770B50446BE
:1048B0000D46164625E02046FFF764FD08B10120AD
:1048C00070BD681CE8B1FDF771FE801BA84200D8DE
:1048D000BDB920684069C0F3C01090B900202063C2
:1048E000202084F83D00002084F83E00206C40F039
:1048F0002000206400BF002084F83C0000BF01209D
:10490000DEE720684069C0F3C0100028D3D0002043
:10491000D6E7000010B501F0C3F84FF480620849F3
:104920000848FFF786F908A000F018F84FF4FA607D
:10493000FDF720FD07A000F011F8FCF763FF10BDA4
:10494000100500206804002041542B4346554E3D7D
:10495000310D0A0041540D0A0000000070B50446F4
:104960004FF400711A48FBF765FC002019490880D4
:10497000194908802046FBF790FC86B24FF4FA7381
:10498000324621461548FFF79BFC4FF47A7514E038
:104990001148008800280DDD11A11248FBF755FCD5
:1049A00020B911A10F48FBF750FC00B170BD0020E9
:1049B000094908800120FDF7DDFC281EA5F1010151
:1049C0008DB2E5D121460AA002F074FB00BFEDE7ED
:1049D000900500204E0000204C00002068040020BC
:1049E0004F4B0000100500204552524F520000006E
:1049F0004154C3FCC1EEB3ACCAB13A2025730A00DE
:104A000010B50248FDF7D8FD10BD0000640200207B
:104A1000FEB504460D4616464FF4FA6001232246C1
:104A2000A121CDE9005602900148FDF7ADFEFEBD83
:104A300064020020FEB504460D4616464FF4FA60A7
:104A400001232246A021CDE9005602900348FEF73B
:104A50001FF80520FDF78EFCFEBD0000640200205B
:104A600000B5A1B021A0FFF779FF4FF49670FDF7D4
:104A700081FC22A0FFF772FF4FF49670FDF77AFCDD
:104A800022A0FFF76BFF6420FDF774FC27A0FFF75F
:104A900065FF6420FDF76EFC2CA32EA231A101A8B6
:104AA00002F018FB01A8FFF759FF4FF4FA60FDF779
:104AB00061FC32A034A336A23AA1009001A802F012
:104AC00009FB01A8FFF74AFF4FF47A70FDF752FC8B
:104AD0003CA244A101A802F0FDFA01A8FFF73EFFA5
:104AE0004FF47A70FDF746FC21B000BD41542B51C4
:104AF0004D54444953433D300D0A000041542B515D
:104B00004D54434C4F53453D300D0A0041542B51F9
:104B10004D544346473D22726563762F6D6F646541
:104B2000222C302C302C300D0A00000041542B5127
:104B30004D544346473D226B656570616C697665EF
:104B4000222C302C36300D0A00000000313838336A
:104B5000000000003130312E3133332E3134312E0C
:104B60003136370041542B514D544F50454E3D3056
:104B70002C222573222C25730D0A00006C646862B8
:104B800030383133000000006C64686200000000BF
:104B90004C444D4355323032353031323041303073
:104BA0003031000041542B514D54434F4E4E3D3057
:104BB0002C222573222C222573222C222573220DD0
:104BC0000A0000002F7365727665722F636F6F2F76
:104BD0004C444D4355323032353031323041303033
:104BE0003031000041542B514D545355423D302C2F
:104BF000312C222573222C310D0A000070B5C2B071
:104C0000FA480088002875DDF949FAA002F052FA46
:104C1000FEA1F748FBF719FB00286CD07B21F44874
:104C2000FBF731FB04467D21F148FBF73DFB0546D0
:104C3000002C7DD0002DFCD0A54279D9281B461C24
:104C40004FF4807102A8FBF7F5FA3246214602A81C
:104C5000FBF70DFB0020019001AAEFA102A8FBF7D2
:104C60002FFB012833D10198012804D0022810D04D
:104C700003282AD11BE0012001F0A6FAE9A002F0E6
:104C800019FA0020D94908808021D948FBF7D2FAC7
:104C90001CE0022001F098FAE6A002F00BFA0020D6
:104CA000D24908808021D248FBF7C4FA0EE00320E5
:104CB00001F08AFAE3A002F0FDF90020CB49088058
:104CC0008021CB48FBF7B6FA00E000BF0AE301AA57
:104CD000E0A102A8FBF7F4FA012835D1E048FEF77D
:104CE000B1FDE048007801280AD0022804D003284A
:104CF0000ED109E0FFE2F7E2DB490198086007E026
:104D0000DA490198086003E0D9490198086000BFBA
:104D100000BF01F0E9FC0020FCF7CAFA0020FCF714
:104D20002BFA0020FCF73AFA0020D249086000E094
:104D3000D9E2D1490860CA490968486201F092F88D
:104D4000C748FEF72BFDCDE201AACCA102A8FBF7D4
:104D5000B7FA01281AD1C3480078012808D00228E0
:104D600002D003280CD107E0C7490198086007E08A
:104D7000C6490198086003E0C5490198086000BF72
:104D800000BF01F0B1FC01F06DF8ABE201AAC1A1D6
:104D900002A8FBF795FA01281AD1B2480078012839
:104DA00008D0022802D003280CD107E0BC490198A2
:104DB000086007E0BB490198086003E0BA49019820
:104DC000086000BF00BF01F08FFC01F04BF889E2E2
:104DD00001AAB6A102A8FBF773FA01281AD1A148CB
:104DE0000078012808D0022802D003280CD107E05F
:104DF000B1490198086007E0B0490198086003E0F4
:104E0000AF490198086000BF00BF01F06DFC01F0E0
:104E100029F867E201AAABA102A8FBF751FA012821
:104E20001AD190480078012808D0022802D003281F
:104E30000CD107E0A6490198086007E0A549019850
:104E4000086003E0A4490198086000BF00BF01F0BA
:104E50004BFC01F007F845E201AAA0A102A8FBF76C
:104E60002FFA01281AD17F480078012808D002289B
:104E700002D003280CD107E09B490198086007E0A5
:104E80009A490198086003E099490198086000BFB9
:104E900000BF01F029FC00F0E5FF23E201AA95A183
:104EA00002A8FBF70DFA012815D10198012808D1B5
:104EB00093490870002093490860012000F010FE1B
:104EC00010E201980028A4D18D4908708D4908602E
:104ED00000F006FE06E201AA8BA102A8FBF7F0F99A
:104EE000012806D18B490198086000208549086097
:104EF000F8E101AA88A102A8FBF7E2F9012806D18E
:104F000088490198086000207E490860EAE101AA0A
:104F100085A102A8FBF7D4F9012829D1019801281D
:104F200002D00198002896D1019808B9012000E02C
:104F30000020804908700198012808D100200870DD
:104F40000120FCF7B5F97CA002F0B4F808E00120DC
:104F5000784908700020FCF7ABF97BA002F0AAF8B2
:104F600000202249088080212148FBF763F9B9E13C
:104F700001AA79A102A8FBF7A3F9012822D101987F
:104F8000012802D00198002887D1019808B9012092
:104F900000E00020734908700198012808D1002022
:104FA00008700120FCF7E8F86FA002F083F899E19F
:104FB00001206C4908700020FCF7DEF86EA002F0BA
:104FC00079F88FE101AA70A102A8FBF779F901280D
:104FD0000AD10198012802D00198002888D10198AF
:104FE000012802D10020D5E0E7E0DCE04C00002001
:104FF00010050020BDD3CAD5B5BDB5C4D4ADCABC5B
:10500000CAFDBEDD3A2025730A0000002B514D5425
:10501000524543563A0000007B22583130223A254F
:10502000647D0000C7D0BBBBB5BDB3E5B2DEC4A391
:10503000CABD0A00C7D0BBBBB5BDB9E0B8C8C4A3E0
:10504000CABD0A00C7D0BBBBB5BDD6B1C5C5C4A3D8
:10505000CABD0A007B22583234223A25647D000002
:10506000B802002018010020D4000020B400002065
:10507000940000201C010020200100207B225832D7
:1050800035223A25647D0000D8000020B8000020B9
:10509000980000207B22583534223A25647D000098
:1050A000DC000020BC0000209C0000207B22583542
:1050B00035223A25647D0000E0000020C000002079
:1050C000A00000207B22583536223A25647D00005E
:1050D000EC000020C4000020A40000207B225835F2
:1050E00037223A25647D0000F0000020C80000202F
:1050F000A80000207B22583135223A25647D00002B
:1051000040010020440100207B22583230223A2501
:10511000647D0000480100207B22583231223A256C
:10512000647D00004C0100207B22583132223A2558
:10513000647D000044000020CBAEB1C3C7BFD6C61B
:10514000BFAAC6F40A000000CBAEB1C3C7BFD6C623
:10515000B9D8B1D50A0000007B22583133223A2554
:10516000647D000045000020B7E7BBFA31C7BFD619
:10517000C6BFAAC6F40A0000B7E7BBFA31C7BFD65C
:10518000C6B9D8B1D50A00007B22583134223A255D
:10519000647D0000594908700120FBF7FFFF58A00B
:1051A00001F088FF9EE00120544908700020FBF7C1
:1051B000F5FF57A001F07EFF94E001AA58A102A8D4
:1051C000FBF77EF801280AD10198012802D0019846
:1051D0000028E7D10199C8B2FCF710F882E001AAD3
:1051E00052A102A8FBF76CF8012807D19DED010A36
:1051F000B8EEC00A504880ED000A73E001AA4FA142
:1052000002A8FBF75DF8012807D19DED010AB8EE71
:10521000C00A4D4880ED000A64E001AA4BA102A833
:10522000FBF74EF8012809D10198012801D0019817
:10523000F8B90199C8B2FBF773FF53E001AA46A180
:1052400002A8FBF73DF801281CD10198012811D1D3
:10525000444908700020444908604448007808B96F
:10526000012000E00020414908700199C8B202F015
:1052700057FE37E00199C8B202F052FE00203949CA
:1052800008702FE001AA3AA102A8FBF719F801283B
:1052900003D1019800F032FE24E001AA37A102A850
:1052A000FBF70EF8012803D1019800F02DFE19E05C
:1052B00001AA35A102A8FBF703F8012812D1019831
:1052C000012803D133A001F0F5FE04E0019810B9E4
:1052D00034A001F0EFFE00203A49088080213A48CE
:1052E000FAF7A8FF00BF00BF0020364908808021E0
:1052F0003548FAF79FFF42B070BD0000450000201E
:10530000B7E7BBFA32C7BFD6C6BFAAC6F40A0000C9
:10531000B7E7BBFA32C7BFD6C6B9D8B1D50A0000C5
:105320007B22583138223A25647D00007B22583296
:1053300032223A25647D00005C0100207B22583235
:1053400033223A25647D0000600100207B2258351D
:1053500039223A25647D00007B22583439223A25CF
:10536000647D0000DC010020E0010020DD01002060
:105370007B22583531223A25647D00007B22583546
:1053800032223A25647D00007B22583538223A25A6
:10539000647D0000C6F4B6AFC5E0BEFAC4A3CABDC2
:1053A0000A000000CDA3D6B9C5E0BEFAC4A3CABDA9
:1053B000A3ACC7D0BBBBB5BDD6B1C5C5C4A3CABD20
:1053C0000A0000004C0000201005002070B50646C1
:1053D0000C4615464FF480710E48FAF72BFF0EA2CB
:1053E00014A10C4801F076FE0A48FFF7B7FA4FF413
:1053F0007A732A4621461648FEF762FF4FF47A7305
:10540000012214A11248FEF75BFF6420FCF7B2FFF3
:1054100070BD0000900700202F6465762F636F6FCA
:105420002F4C444D435532303235303132304130DB
:105430003030310041542B514D545055423D302CA9
:10544000302C302C302C222573220D0A0000000055
:10545000680400201A00000010B500F0AFFC0446FC
:105460005C480078844209D000205B4908605B49B1
:10547000086001205A49087056480470002C52D127
:105480005848007830B10020FBF712FF0020564941
:1054900008601FE05048006854490968884206D2F5
:1054A0000120FBF705FF01204F49086012E04F483B
:1054B00000684F490968084447490968884206D985
:1054C0000020FBF7F5FE00204749086002E00020BD
:1054D000414908604748007818B10020FBF770FE8A
:1054E00077E03E48006844490968884203D20120B9
:1054F000FBF766FE6DE00020FBF762FE3E480068A9
:105500003E490968084435490968884261D8002045
:10551000324908603A48007808B9012000E00020CC
:105520003749087055E00020FBF7C2FE00202E49E5
:1055300008603048007818B10020FBF741FE48E0D1
:105540002748007820B3254800682E49096888421A
:1055500003D20120FBF734FE3BE00020FBF730FED6
:10556000284800682849096808441C490968884295
:105570002FD80020194908602148007808B9012077
:1055800000E000201E49087000201549087020E046
:10559000124800681D490968884203D20120FBF7C0
:1055A0000FFE16E00020FBF70BFE184800681849B4
:1055B000096808440949096888420AD8002007494F
:1055C00008600F48007808B9012000E000200C496D
:1055D000087010BD310100201C01002020010020B6
:1055E00025010020440000202C010020D4000020D0
:1055F000D800002045000020DC000020E000002052
:1056000024010020E4000020E8000020EC0000203D
:10561000F000002000B58DB0002009900A900B909A
:105620000C90202101A8FAF705FE214821490860C5
:105630000020486000211F4881600161017680F8E8
:105640002010C1621C4981620021C1600121C16139
:10565000002180F8301001214161FCF7E5FA08B122
:10566000FBF7EAFF0420099001200A9006200B9026
:1056700009A91048FCF70EFA08B1FBF7DDFF04207A
:1056800001900120029005900020039008900B48A3
:10569000079000208DF819008DF81800049001A9DA
:1056A0000448FCF7E3F808B1FBF7C6FF0DB000BDF6
:1056B000002201401C0200200100000F01000F0029
:1056C00008B500BF002000900A48006840F40010B0
:1056D000084908600846006800F40010009000BF08
:1056E00000BF002211460D20FDF750FB0D20FDF7F5
:1056F00039FB08BD3038024000B587B0142102A83C
:10570000FAF798FD00BF002001905548006840F06E
:105710001000534908600846006800F0100001902E
:1057200000BF00BF00BF002001900846006840F0A5
:10573000040008600846006800F00400019000BF03
:1057400000BF00BF002001900846006840F0200024
:1057500008600846006800F02000019000BF00BF0C
:1057600000BF002001900846006840F080000860FB
:105770000846006800F08000019000BF00BF00BF35
:10578000002001900846006840F0010008600846CB
:10579000006800F00100019000BF00BF00BF0020C2
:1057A00001900846006840F0400008600846006824
:1057B00000F04000019000BF00BF00BF002001903A
:1057C0000846006840F0080008600846006800F0DD
:1057D0000800019000BF00BF00220C212148FCF707
:1057E000DFFE002242F65E211F48FCF7D9FE0C20A6
:1057F00002900120039000200490059002A919480E
:10580000FCF7CCFD0420029000200390049002A934
:105810001648FCF7C3FD20200290002003900120D1
:10582000049002A91248FCF7B9FD40F61E20029030
:105830000120039000200490059002A90A48FCF77B
:10584000ADFD4FF401500290012003900020049020
:105850000220059002A90448FCF7A0FD07B000BD96
:10586000303802400010024000180240001402408C
:105870000008024010B50B480B4908600B4848600F
:10588000002109488160C1604FF48041016100211D
:1058900041618161C1610162FCF78EFE08B1FBF7D5
:1058A000CBFE10BD0058004064020020A08601001D
:1058B00000B587B0002003900490059006900190F9
:1058C00002904FF080401449086041F61F40486044
:1058D0000021114881601149C1600021016181618D
:1058E000FDF7AAFE08B1FBF7A7FE4FF48050039026
:1058F00003A90948FDF7C5FF08B1FBF79DFE00208D
:105900000190029001A90448FDF73CFE08B1FBF7A5
:1059100093FE07B000BD0000B8020020BF270900B9
:1059200000B587B000200390049005900690019088
:10593000029015481549086041F61F404860002153
:105940001248816042F20F71C160002101618161E2
:10595000FDF772FE08B1FBF76FFE4FF48050039025
:1059600003A90A48FDF78DFF08B1FBF765FE00208B
:105970000190029001A90548FDF704FE08B1FBF76C
:105980005BFE07B000BD00000004004000030020E3
:105990001CB50020009001900E480F490860472078
:1059A000486000210C48816040F2E731C16000216D
:1059B0008161FDF741FE08B1FBF73EFE002000903B
:1059C000019069460448FDF7DDFD08B1FBF734FEA0
:1059D0001CBD000000100040480300201CB5002042
:1059E000009001900E480F49086041F61F40486042
:1059F00000210C48816042F20F71C1600021816179
:105A0000FDF71AFE08B1FBF717FE00200090019089
:105A100069460448FDF7B6FD08B1FBF70DFE1CBD55
:105A2000001400409003002010B50D480D49086097
:105A30004FF4965048604FF480510A48816000212D
:105A4000C1604FF4806101610C21416100218161DD
:105A5000C161FEF7B5FA08B1FBF7EEFD10BD00001D
:105A6000004C0040D803002010B50B480B490860DB
:105A70004FF4E1304860002108488160C160016155
:105A80000C21416100218161C161FEF799FA08B1E1
:105A9000FBF7D2FD10BD00000010014020040020E3
:105AA00010B50B480B4908604FF4E1304860002105
:105AB00008488160C16001610C2141610021816160
:105AC000C161FEF77DFA08B1FBF7B6FD10BD00001D
:105AD000004400406804002000BFFEE700BFFEE76E
:105AE00010B504462CB1012240210548FCF758FDB1
:105AF00004E0002240210248FCF752FD10BD0000E6
:105B00000018024010B512480078E8B1114800684A
:105B100011490968884203D80120FFF7E1FF16E028
:105B20000D4800680D49096808440A490968884217
:105B300003D30020FFF7D4FF09E0002005490860E7
:105B40000120FFF7CDFF02E00020FFF7C9FF10BDE5
:105B50004001002044010020480100204C010020A9
:105B600010B540210148FCF713FD10BD001802409C
:105B700010B5012004490870002004490860012084
:105B8000FFF7AEFF10BD00004001002044010020DF
:105B90007047000010B500F05DF9044694B1154857
:105BA000007878B901201349087000201249086074
:105BB0001248007808B9012000E000200F49087061
:105BC000FBF73EFB0B48007890B10B480068401C87
:105BD000094908600846006809490968884207D3EE
:105BE0000020FBF71BFB00200249087002490860F7
:105BF00010BD0000DC010020E0010020DD010020DC
:105C0000E401002010B52DED0E8B9FED4A0AF0EE59
:105C1000408A4948FCF7E4F864214748FCF778F8E3
:105C2000002871D14448FBF7FBFF4449088008462F
:105C3000008800EE100AB8EE400ADFED410A20EEBF
:105C4000200ADFED3C0A20EE200A3E4880ED000AE3
:105C500090ED000ADFED3C0A20EE200AD0ED000AAC
:105C60009FED3A1A71EE600A80EE201AB0EE418A7A
:105C70009FED350AC8EE000A10EE904A2046FAF76A
:105C800069FD41EC1E0BB0EE4E0AF0EE6E0A01F01B
:105C900053FAB0EE40DAF0EE60DA9FED2D0B53ECE4
:105CA000102B51EC1D0BFAF7E6FC41EC1C0B9FEDA1
:105CB0002A0B53EC102BFAF7C5FB41EC1B0B53ECF2
:105CC0001B2B9FED270B51EC100BFAF7D4FC41EC8A
:105CD0001A0B9FED250B53EC102BFAF754FC41ECFB
:105CE000190BFAF763FD22490860084690ED000A97
:105CF0002048D0ED000AB4EEE00AF1EE10FA04D22A
:105D00000120FBF77BFA0EE00EE0194890ED000A47
:105D10001948D0ED000AB4EEE00AF1EE10FA02DD07
:105D20000020FBF76BFA00BF0348FCF7FFF8BDEC5F
:105D30000E8B10BD9A99193F1C02002064010020AF
:105D40003333533A6801002000401C46333353403C
:105D50000000000000DCAE40000000E0E1796B3F95
:105D6000000000000000F03F00000060661271407B
:105D70006C0100205C0100206001002010B51021A2
:105D80000148FCF705FC10BD0018024010B50421C5
:105D90000148FCF7FDFB10BD0018024010B50821BA
:105DA0000148FCF7F5FB10BD0018024010B520219A
:105DB0000148FCF7EDFB10BD0008024010B5FFF7ED
:105DC000F5FF04460E480078844205D000200D49B6
:105DD00008700B48047010E00A4800780A280CDAB2
:105DE00008480078401C07490870084600780A28CF
:105DF00003DB05480470002008700348007810BDDC
:105E000027010020260100202801002010B54FF4B2
:105E100000710248FCF7BCFB10BD000000180240F6
:105E200010B504210148FCF7B3FB10BD001402407B
:105E300010B504210648FCF7ABFB20B90821044843
:105E4000FCF7A6FB08B1012010BD0020FCE7000014
:105E50000010024010B502210148FCF799FB10BD6B
:105E60000018024010B51B48FDF7ECFC00F082F969
:105E70000020194908601949086019490860194942
:105E80000860012018490870002018490860184966
:105E900008704FF47A70FCF76DFA16480078012804
:105EA00004D0022805D0032809D105E000F0D0F97C
:105EB00005E000F0EDF902E000F0B0F900BF00BF2E
:105EC000002005490860054908600248FDF766FCA6
:105ED00010BD0000B80200201C010020200100209D
:105EE0001001002014010020250100202C010020B9
:105EF00024010020180100207047000001490860BB
:105F000070470000E401002001490860704700006C
:105F1000E801002010B5FFF751FF044680480078E3
:105F2000844207D000207F49086001207E49087024
:105F30007B48047014BB7B4800687C490968884230
:105F400003D20120FBF73CF963E078480068784908
:105F50000968084473490968884203D90020FBF79F
:105F60002FF956E000206F4908607248007808B9A0
:105F7000012000E000206F4908704AE06A4800787C
:105F800028B3684800686C490968884203D2012038
:105F9000FBF716F93DE0684800686849096808445D
:105FA00060490968884203D90020FBF709F930E00D
:105FB00000205C4908605F48007808B9012000E0D3
:105FC00000205C49087000205749087021E05548BE
:105FD00000685B490968884203D20120FBF7F0F8AA
:105FE00017E0574800685749096808444D4909684F
:105FF000884203D90020FBF7E3F80AE00020494972
:1060000008604C48007808B9012000E000204949A8
:1060100008704D48007830B1012819D0022847D0C7
:1060200003287BD174E00020FBF742F900204749A8
:1060300008604748006847490968884207D9012035
:10604000414908700020424908604349086065E002
:106050003F48006841490968884220D23E480068AC
:106060003F490968884206D20120FBF721F9012047
:10607000364908601BE03A4800683A490968084414
:1060800035490968884206D90020FBF711F900203C
:106090002E4908600BE000202F49086007E002202D
:1060A0002949087000202A4908602B49086035E01A
:1060B000274800682C490968884220D22648006891
:1060C00027490968884206D20120FBF7F1F8012030
:1060D0001E4908601BE022480068244909680844FA
:1060E0001D490968884206D90020FBF7E1F8002025
:1060F000164908600BE000201749086007E00320FC
:106100001149087000F08AF803201949087005E069
:1061100000F084F803201649087000BF00BF10BDCE
:106120003301002020010020250100209C000020D8
:10613000A000002024010020AC000020B0000020BE
:10614000A4000020A80000200C0100202C01002049
:1061500010010020F400002014010020F8000020AD
:10616000FC000020000100200401002008010020A4
:106170001801002010B50020FBF79AF80020FAF76C
:10618000FBFF0020FBF70AF80020094908600949D5
:106190000860094908600949086001200849087039
:1061A0000020084908604FF47A70FCF7E3F810BD4E
:1061B0001C010020200100201001002014010020FB
:1061C000250100202C01002010B50446FFF7D2FF66
:1061D000012C06D0022C0AD0032C0ED0042C18D18E
:1061E00011E000F035F801200B49087012E000F0D2
:1061F0004FF80220084908700CE000F00FF8032067
:106200000549087006E000F063F8042002490870B0
:1062100000E000BF00BF10BD1801002010B5002035
:106220000849086008490860FFF7C8FD0749087079
:106230000020FBF73DF80020FAF79EFF0020FAF758
:10624000ADFF10BD1C010020200100203001002006
:1062500010B500200A4908600A49086001200A496F
:106260000870FFF7ABFD094908700020FBF720F824
:106270000020FAF781FF0020FAF790FF10BD000020
:106280001C010020200100202501002032010020F7
:1062900010B500200A4908600A49086001200A492F
:1062A0000870FFF78BFD094908700020FBF700F824
:1062B0000020FAF761FF0020FAF770FF10BD000020
:1062C0001C010020200100202501002031010020B8
:1062D00010B500200D4908600D4908700D4908608F
:1062E0000D49086001200D490870FFF767FD0C4952
:1062F00008700020FAF7DCFF0020FAF73DFF0020CD
:10630000FAF74CFF04200749087010BD2001002057
:106310000C010020100100201401002025010020A4
:10632000330100201801002010B5FCF7A7FC10BDB8
:1063300000B593B0302107A8F9F77CFF142102A81B
:10634000F9F778FF00BF002001902348006840F073
:106350008050214908600846006800F08050019094
:1063600000BF00BF00BF002001901C48006840F43F
:1063700080401A4908600846006800F48040019097
:1063800000BF00BF012007900004089002200D907C
:1063900041050E9108210F91902110910221119138
:1063A0000421129107A8FCF783FE08B1FBF744F91A
:1063B0000F20029002200390002004904FF48050A0
:1063C000059000200690022102A8FCF731FD08B1DB
:1063D000FBF732F913B000BD4038024000700040B6
:1063E0000348006840F470000149086070470000ED
:1063F00088ED00E010B50248FDF7CAFA10BD0000B4
:10640000B802002010B50248FDF7C2FA10BD000026
:106410000003002010B50248FDF7BAFA10BD0000D5
:106420004803002010B50248FDF7B2FA10BD000085
:106430009003002010B502682D4B98420ED0B0F1A9
:10644000804F0BD02B4B984208D02B4B984205D055
:106450002A4B984202D02A4B984203D122F0700274
:106460004B681A43224B984220D0B0F1804F1DD088
:10647000204B98421AD0204B984217D01F4B98427D
:1064800014D01F4B984211D01E4B98420ED01E4B79
:1064900098420BD01D4B984208D01D4B984205D016
:1064A0001C4B984202D01C4B984203D122F44072FC
:1064B000CB681A4322F080034C6943EA040202606D
:1064C0008B68C3620B688362094B984202D00C4B05
:1064D000984201D10B69036301234361036903F00F
:1064E00001031BB1036923F00103036110BD000028
:1064F000000001400004004000080040000C004083
:1065000000040140004001400044014000480140B7
:1065100000180040001C00400020004030B50C4630
:10652000816821F47F4142EA0325254329438160A4
:1065300030BD0A46816821F0700142F0070319431B
:106540008160704730B50B461446026A056A25F033
:1065500001050562816921F0F00141EA041122F090
:106560000A021A438161026230BD30B50B461446FF
:10657000026A056A25F010050562816921F47041FF
:1065800041EA043122F0A00242EA03128161026270
:1065900030BD000010B504223B490020FEF738FA58
:1065A00004223A491046FEF733FA042238490820FB
:1065B000FEF72EFA042237490C20FEF729FA0422AE
:1065C00035491020FEF724FA042234491420FEF73E
:1065D0001FFA042232491820FEF71AFA0422314920
:1065E0001C20FEF715FA04222F492020FEF710FA8E
:1065F00004222E492420FEF70BFA04222C492820DD
:10660000FEF706FA04222B492C20FEF701FA042299
:1066100029493020FEF7FCF9042228493420FEF7EE
:10662000F7F9042226493820FEF7F2F90422254919
:106630003C20FEF7EDF9042223494020FEF7E8F95B
:10664000042222494420FEF7E3F90422204948208D
:10665000FEF7DEF904221F494C20FEF7D9F9042287
:106660001D495020FEF7D4F904221C495420FEF79E
:10667000CFF904221A495820FEF7CAF90422194911
:106680005C20FEF7C5F910BD9400002098000020A2
:106690009C000020A0000020A4000020A8000020F2
:1066A000AC000020B0000020B4000020B8000020A2
:1066B000BC000020C0000020C4000020C800002052
:1066C000CC000020D0000020D4000020D800002002
:1066D000DC000020E0000020EC000020F0000020A2
:1066E000E4000020E800002010B504223B4900200F
:1066F000FEF7A0F904223A491046FEF79BF904225E
:1067000038490820FEF796F9042237490C20FEF795
:1067100091F9042235491020FEF78CF904223449FE
:106720001420FEF787F9042232491820FEF782F977
:10673000042231491C20FEF77DF904222F49202034
:10674000FEF778F904222E492420FEF773F904227B
:106750002C492820FEF76EF904222B492C20FEF745
:1067600069F9042229493020FEF764F904222849F6
:106770003420FEF75FF9042226493820FEF75AF943
:10678000042225493C20FEF755F9042223494020E4
:10679000FEF750F9042222494420FEF74BF9042267
:1067A00020494820FEF746F904221F494C20FEF7F5
:1067B00041F904221D495020FEF73CF904221C49EE
:1067C0005420FEF737F904221A495820FEF732F90F
:1067D000042219495C20FEF72DF910BD9400002019
:1067E000980000209C000020A0000020A4000020B1
:1067F000A8000020AC000020B0000020B400002061
:10680000B8000020BC000020C0000020C400002010
:10681000C8000020CC000020D0000020D4000020C0
:10682000D8000020DC000020E0000020EC00002068
:10683000F0000020E4000020E800002010B502482D
:10684000FDF74AFA10BD0000D803002070B50546D8
:10685000AC6B0020E085E0842046FDF73BFA70BD7C
:1068600000BF00BF02680C3252E8002F22F4907182
:1068700002680C3242E80013002BF3D100BF00BFC6
:1068800000BF0268143252E8002F22F001010268B2
:10689000143242E80013002BF3D100BF016B012931
:1068A0000ED100BF00BF02680C3252E8002F22F068
:1068B000100102680C3242E80013002BF3D100BF34
:1068C000202180F8421000210163704710B5044672
:1068D0002068C06820F040002168C860202084F84B
:1068E00041002046FDF74BFD002010BDF8B50446E1
:1068F00094F84200222875D1A068B0F5805F0CD1D1
:10690000206950B90025A66A20684068C0F30800D5
:106910003080A06A801CA06215E0A56A0026A068ED
:10692000B0F5805F03D0A06828B9206918B9206845
:106930004068287004E02068406800F07F002870FC
:10694000A06A401CA062E08D401E80B2E085002855
:1069500046D12068C06820F020002168C860206807
:10696000C06820F480702168C8602068406920F009
:10697000010021684861202084F842000020606303
:10698000206B012826D10020206300BF00BF2168B2
:106990000C3151E8001F21F0100021680C3141E852
:1069A0000002002AF3D100BF2068006800F0100048
:1069B00010280AD100BF00200090206800680090D5
:1069C00020684068009000BF00BFA18D2046FDF701
:1069D00069F902E02046FDF72FFC0020F8BD01E038
:1069E0000020FBE70220F9E72DE9F84F0446206874
:1069F000006920F44050E16808432168086121697A
:106A0000A068084361690843E16908430090206871
:106A1000C06849F20C618843009908432168C86046
:106A20002068406920F44070A169084321684861EA
:106A300076492068884203D075492068884203D18E
:106A4000FCF7CEFA814602E0FCF7BAFA8146E0692B
:106A5000B0F5004F6CD102206168A0FB01500346E5
:106A60001920A9FB007001462A463846F9F7AAFB0F
:106A70006421B0FBF1F04FEA001A02206168A0FB2C
:106A800001510B461920A9FB00712A463846F9F737
:106A900099FB834602206168A0FB01500346192040
:106AA000A9FB00712A463846F9F78CFB6421B0FB3C
:106AB000F1F000EBC00101EB0010ABEB80003221E4
:106AC00001EBC0006421B0FBF1F000F0F8000AEB2C
:106AD000400A02206168A0FB015003461920A9FB6F
:106AE000007001462A463846F9F76CFB83460220BF
:106AF0006168A0FB015003461920A9FB00712A46DA
:106B00003846F9F75FFB6421B0FBF1F000EBC00100
:106B100001EB0010ABEB8000322101EBC0006421DF
:106B2000B0FBF1F000F007005044216888606AE093
:106B300004206168A0FB015003461920A9FB0070E6
:106B400001462A463846F9F73DFB82460420616833
:106B5000A0FB015003461920A9FB007001462A46FC
:106B60003846F9F72FFB6421B0FBF1F000EBC001D0
:106B700001EB0010AAEB8000322101EB0010642130
:106B8000B0FBF1F000F0F00A04206168A0FB017096
:106B900003461920A9FB00513A462846F9F712FB93
:106BA0006421B0FBF1F00AEB001A04206168A0FB3D
:106BB00001510B461920A9FB00712A463846F9F706
:106BC00001FB834604206168A0FB015003461920A5
:106BD000A9FB007001462A463846F9F7F3FA64210A
:106BE000B0FBF1F000EBC00101EB0010ABEB80005B
:106BF000322101EB00106421B0FBF1F000F00F0036
:106C0000504421688860BDE8F88F00000010014002
:106C10000014014010B5034699629A85DA85002078
:106C20005864222083F84200186928B11868C068A7
:106C300040F480701C68E0601868406940F0010012
:106C40001C6860611868C06840F020001C68E06043
:106C5000002010BD014691F84100212828D1886804
:106C6000B0F5805F0BD1086948B90A6A1088C0F393
:106C700008000B685860086A801C086205E00B6A0F
:106C8000581C086218780B685860C88C401E80B287
:106C9000C88458B90868C06820F080000B68D860C4
:106CA0000868C06840F040000B68D860002070475A
:106CB0000220FCE72DE9F84304460D4617469846A6
:106CC000089E31E0701C70B3FBF770FCA0EB08006D
:106CD000B04200D816B90320BDE8F8832068C06828
:106CE00000F00400F8B1802D1ED0402D1CD020688B
:106CF0000068C0F3C000B0B100BF00200090206861
:106D00000068009020684068009000BF00BF2046E7
:106D1000FFF7A6FD0820606400BF002084F8400053
:106D200000BF0120D8E7FFE7206800682840A8429C
:106D300001D1012000E00020B842C3D00020CBE701
:106D400010B50248FCF7C8FF10BD00006804002021
:106D500010B51448007814490870FFF77BF8124901
:106D60004870FFF713F810498870FFF717F80E49BD
:106D7000C870FEF7F5FE0C490871FFF717F80A49CD
:106D80004871FFF743F80849C871FFF749F8064909
:106D90000872FFF74DF804494872FEF7EFFF024909
:106DA000887210BD68000020900800202DE9F0478F
:106DB0002DED068BE2B0FFF7CBFFFAF77FF9FEF778
:106DC00021FFFAF71FFD002500260027A846A94647
:106DD000AA4671480078012816D0022804D003285A
:106DE00022D0042860D12FE06C4805686C48066802
:106DF0006C4807686C48D0F800806C48D0F8009068
:106E00006B48D0F800A04FE06A4805686A480668F9
:106E10006A4807686A48D0F800806A48D0F800904D
:106E20006948D0F800A03FE06848056868480668EF
:106E3000684807686848D0F800806848D0F8009033
:106E40006748D0F800A02FE0624807686248D0F891
:106E500000806248D0F800906148D0F800A06148F6
:106E6000007820B1012809D0022817D10EE05EA0D9
:106E700000F020F900256448066813E063A000F0E4
:106E800019F96A4805686A4806680BE069A000F0CD
:106E900011F9664805686F48066803E06EA000F0C7
:106EA00009F900BF00BF00BF00BF72480068F9F7D2
:106EB00051FC41EC180B70480068F9F74BFC41ECB1
:106EC000190B6E480068F9F745FC41EC1A0B6C4849
:106ED00090ED000B8DED200B2F480078042801D198
:106EE000012000E00020CDE91D9ACDF870801F90B0
:106EF0006448807A64490968644A1268CDE91A07CF
:106F0000CDE918215F48407A61490A7861490B78D8
:106F10005C49097ACDE915321491179059484079A6
:106F20005D4989785C4A52785B4B1B78CDE90E56F7
:106F3000CDE91032CDE912108DED0C8B8DED0A9B51
:106F40008DED08AB55480168554802684D48C07939
:106F5000544B1B78CDE90330CDE905214948C07871
:106F600048498978474A5278CDE9002102900A4879
:106F700003784D4890F900204C4922A800F0AAF867
:106F800084B2224622A90020FEF720FA62B0BDECAE
:106F9000068BBDE8F087000018010020D400002017
:106FA000D8000020DC000020E0000020EC000020E1
:106FB000F0000020B4000020B8000020BC00002039
:106FC000C0000020C4000020C80000209400002061
:106FD000980000209C000020A0000020A4000020B9
:106FE000A80000200C010020CCD8CAE2C4A3CABD6E
:106FF000B3F5CABCBDD7B6CE202D203234D0A1CA3D
:10700000B1CDA3D6B90A0000F4000020CCD8CAE262
:10701000C4A3CABDB5DAD2BBBDD7B6CE202D2036AB
:10702000D0A1CAB1D1ADBBB70A000000FC0000205E
:1070300000010020CCD8CAE2C4A3CABDB5DAB6FEAE
:10704000BDD7B6CE202D2034D0A1CAB1D1ADBBB7AB
:107050000A00000008010020B4EDCEF3A3BACEDE92
:10706000D0A7B5C4CCD8CAE2C4A3CABDBDD7B6CEDA
:107070000A000000600100205C0100206C0100207B
:10708000B801002090080020E8010020E401002061
:10709000EC010020FC0100207D0000204C010020BC
:1070A00048010020400100205100002078810008A4
:1070B00000BFFEE70FB4054B10B503A9044A0298C0
:1070C00000F0A6FB10BC5DF814FB0000497F00082F
:1070D000140200200FB4084B10B504A902AA0398AB
:1070E00000F096FB044602A9002000F014FF2046A1
:1070F00010BC5DF814FB0000177F00080248006810
:10710000C0F30220704700000CED00E010B500282D
:1071100004DB0A07130E054A135406E00A07140E8F
:10712000034A00F00F031B1FD45410BD00E400E01D
:1071300018ED00E00000000070B5D94B00242DEDE3
:10714000020B2DED108BDDE91010984205DA20F0CE
:1071500000429A4201D809D141B19DED100BBDEC1E
:10716000108B02B0BDE8704000F05EBAB0F5801F31
:1071700026DA11430BD0002813DA012000F080FA40
:10718000BDEC108B02B0BDE8704000F059BA02208F
:1071900000F076FA00F030FA51EC100B81F000416B
:1071A0009EE06FF035049FEDC00B53EC102B9DED6E
:1071B000100B51EC100BF9F7ECF9CDE91001084672
:1071C00004EB2051C0F31304B948A1F2FF3120446D
:1071D00000F4801080F07F6282F04052224301EB85
:1071E00020559FEDB50B119253EC102B9DED100B1C
:1071F00051EC100BF9F7C7F941EC180BA01CC0F3C8
:1072000013009FEDAFDB9FEDB0EBB14E7E44032842
:107210006CD296ED000B51EC180B53EC102BF9F7D8
:1072200029FC1DD1002D01BF96ED000BBDEC108B8C
:1072300002B070BD2846F9F7F3FB41EC180B53EC94
:107240001D2BF9F7A6F941EC190B53EC1E2B51EC51
:10725000180BF9F79EF953EC192BF9F7F3F83FE007
:107260009FED9D0B51EC180B53EC102BF9F791F996
:107270009FED9B1B53EC112BF9F788F941EC190B8F
:1072800053EC182B51EC180BF9F783F953EC192B2D
:10729000F9F77FF941EC190B002D04BF53EC192BC2
:1072A00051EC180B1AD02846F9F7BAFB41EC1A0B2F
:1072B00053EC1D2BF9F76DF953EC192BF9F766F91F
:1072C00053EC182BF9F75FF941EC180B53EC1E2B1C
:1072D00051EC1A0BF9F75DF953EC182BF9F753F948
:1072E000BDEC108B02B041EC100B70BD9FED7E0B1E
:1072F00051EC180B53EC102BF9F7A4F841EC100BE0
:1073000051EC180B53EC102BF9F7B5F941EC190BB4
:107310002846F9F785FB41EC1B0B53EC192B51EC7C
:10732000190BF9F736F941EC1A0B714853EC1A2B8B
:10733000261851EC1A0BF9F72CF941EC1F0B6D488C
:10734000C4F1510404F5D724B0EE4F0AF0EE6F0AF1
:107350000321784400F0D2F853EC1F2B51EC100BB2
:10736000F9F717F941EC1C0B6348B0EE4F0AF0EE49
:107370006F0A0421784400F0C1F853EC1A2B51EC49
:10738000100BF9F706F9344353EC1C2BF9F75AF8B4
:1073900041EC1C0B002C4CDD9FED510B51EC180BFC
:1073A00053EC102BF9F7F5F853EC182BF9F7F1F82B
:1073B00041EC1A0B55B353EC1D2B51EC1B0BF9F799
:1073C000E8F841EC1D0B53EC1C2B51EC1A0BF9F7B0
:1073D00039F853EC192BF9F7DCF853EC1D2BF9F7BE
:1073E00031F853EC1A2BF9F7D1F853EC182BF9F7C5
:1073F000CAF841EC180B53EC1E2B51EC1B0BF9F7A0
:10740000C8F853EC182BF9F7BEF869E753EC1C2BBE
:1074100051EC1A0BF9F716F853EC192BF9F7B9F8E8
:1074200053EC1A2BF9F7B2F853EC182BF9F7AEF826
:1074300056E735B353EC1D2B51EC1B0BF9F7A9F8AC
:1074400041EC1A0B53EC1C2B51EC180BF9F79BF881
:1074500053EC192BF9F79DF853EC1A2BF9F793F825
:1074600053EC182BF9F78FF841EC180B53EC1E2B4B
:1074700051EC1B0BF9F78DF853EC182BF9F783F847
:107480002EE753EC1C2B51EC180BF9F77CF853EC5E
:10749000192BF9F77EF853EC182BF9F777F81FE75B
:1074A0000000F07F000000000000000000005043DA
:1074B000645F090000000000000000000000F03FD1
:1074C000763C7935EF39EA3D0000E0FE422EE63F9A
:1074D000200F000000000000555555555555D53F6B
:1074E000000000000000E03F00000000000000403D
:1074F00086EBF9FFA20D0000980D000070B5044660
:107500002DED028B4D1E00EBC500B0EE408AF0EE73
:10751000608A90ED000B35F0060017D053EC182B65
:1075200051EC100BF9F735F841EC100B6D1E04EB24
:10753000C50090ED001B51EC100B53EC112BF8F72C
:1075400081FF41EC100B35F00600E7D1022D36D05B
:10755000042D1CD0062D1CBFBDEC028B70BD53EC5E
:10756000182B51EC100BF9F714F894ED0A1B53EC9F
:10757000112BF8F767FF53EC182BF9F70AF894ED85
:10758000081B53EC112BF8F75DFF41EC100B53EC8B
:10759000182B51EC100BF8F7FCFF94ED061B53EC85
:1075A000112BF8F74FFF53EC182BF8F7F2FF94ED7F
:1075B000040B53EC102BF8F745FF41EC100B53EC88
:1075C000182B51EC100BF8F7E4FF94ED021B53EC71
:1075D000112BF8F737FF53EC182BF8F7DAFF94ED7F
:1075E000001B53EC112BF8F72DFFBDEC028B41EC87
:1075F000100B70BD000000009FED070B10B553ECA1
:10760000102B9FED070B51EC100BF9F734F841EC00
:10761000100B10BD00000000000000000000000082
:10762000000000000000F03F10B553EC102B51ECAF
:10763000100BF8F707FF41EC100B10BD0000000025
:107640009FED050B10B553EC102B51EC100BF9F717
:1076500012F841EC100B10BD00000000000000000B
:1076600002E008C8121F08C1002AFAD1704770470B
:10767000002001E001C1121F002AFBD17047000069
:107680000149086070470000180200202DE9FF5FE3
:1076900082B00021DDE90430020DDDF840B0034383
:1076A00018D044F61050A2F2FF324243151411983C
:1076B00001281FD0A5EB0B00401C5FEA000A4FF029
:1076C00000064E4FDFF83891B046504615D5CAF146
:1076D000000413E0119801244AA3012801D16FEAA4
:1076E0000B010298119AC0E90031C0E9024206B0CC
:1076F000BDE8F09FCBF10000DFE704460021404ADF
:10770000491842EB0450CDE9001012E0E00707D021
:1077100032463B4640464946F8F73BFF804689469D
:1077200032463B4610461946F8F733FF06460F46E9
:107730006410002CEAD1DDE90401DDE90023BAF18F
:10774000000F06DAF8F725FF42464B46F8F721FF0F
:1077500005E0F8F790FF42464B46F8F78CFF0446E9
:107760000E460022284BF9F709F803D84FF0FF30F6
:10777000014607E00022254B20463146F8F762FE1D
:10778000F9F75FF9102409E0002C0ADB0A22002334
:10779000F8F718FD039B30321A55641E50EA0102B7
:1077A000F2D1641C039AC4F111031444119A012A02
:1077B00003D0012208430DD10AE0084304D0002081
:1077C0004FF0110B119072E7A3EB0B056D1E0DE04E
:1077D0005B4504DD4FF0000205F1010504E003DA2A
:1077E0004FF00002A5F10105002AECD00298119992
:1077F000C0E90231C0E9004579E70000000014400B
:107800000000F03F300000000000F0430000E03FC7
:107810002DE9FF4F95B09A46884606460025EEE1D1
:10782000252877D100242746F94A0121039400E056
:10783000044316F8013F203B01FA03F01042F7D150
:1078400030782A2811D06FF02F033078A0F1300261
:10785000092A16D8039A44F0020402EB820203EBD1
:1078600042021044761C0390EFE758F8042B039271
:10787000002A03DA504244F40054039044F0020416
:10788000761C30782E2816D116F8010F44F0040427
:107890002A280DD06FF02F023078A0F13003092B89
:1078A00009D807EB870302EB4303C718761CF3E7FD
:1078B00058F8047B761C30786C280FD006DC4C28F6
:1078C00017D068280DD06A2814D104E0742810D08D
:1078D0007A280FD10DE044F400140AE044F4801437
:1078E00001E044F440147278824202D104F580141D
:1078F000761C761C307866280BD013DC582877D09D
:1079000009DC002875D04528F6D04628F4D0472851
:107910001AD193E118E0632835D0642879D065281E
:1079200012D18BE1702873D008DC6728F1D0692868
:107930006FD06E280DD06F2806D1ACE073282CD004
:10794000752874D0782853D05246179990476D1CEB
:1079500054E1C4F30250022809D003280DD0D8F80E
:10796000001004280DD00D6008F1040846E1D8F895
:107970000010EA17C1E90052F6E7D8F800100D80B0
:10798000F2E70D70F0E718F8041B8DF800100020E6
:107990008DF80100EB46012003E058F804BB4FF0DE
:1079A000FF3061074FF0000102D40DE009F1010141
:1079B0008946B9420FDA8145F8DB1BF80910002926
:1079C000F4D108E009F1010189468142FADB1BF894
:1079D00009100029F6D103985346A0EB0907214668
:1079E0003846179A00F080FA284400EB090507E0B2
:1079F00044E008E10DE01BF8010B5246179990474F
:107A0000B9F10109F7D2534621463846179AF2E0F8
:107A100039E00A21C4F302524FF0000B0091022A10
:107A200006D058F8040BC117032A09D00AE023E056
:107A300008F1070020F00702F2E80201904605E095
:107A400000B2C117042A01D140B2C117002906DAD9
:107A50000A460021404261EB02012D2202E022058C
:107A600004D52B228DF80420012203E0E20701D087
:107A70002022F7E7914657E00A2100E010214FF05D
:107A8000000B00910BE010214FF0000B44F00404B8
:107A90000827009103E008204FF0000B0090C4F38A
:107AA0000252022A05D058F8040B0021032A08D0FC
:107AB00008E008F1070020F00702F2E80201904612
:107AC00003E080B2042A00D1C0B24FF000092207BF
:107AD0002AD53278702A07D0DDF800C08CF0100C5F
:107AE0005CEA0B0C05D00EE040228DF80420012248
:107AF00008E050EA010306D030238DF804308DF8F9
:107B0000052002229146009B83F0080353EA0B03F1
:107B10000AD150EA010201D1620705D530228DF861
:107B200004204FF001097F1E3278582A04D039A270
:107B30000C920CAA02920BE03BA2F9E75B46009A7A
:107B4000F8F740FB0C9B9B5C029A521E029213704A
:107B500050EA0102F2D1029804A9081A00F1200BA0
:107B6000600702D524F4803400E001275F4502DD80
:107B7000A7EB0B0000E0002000EB0B010090039846
:107B80004944401A0390E00306D453462146179A0D
:107B9000039800F0A9F90544002706E001A8524621
:107BA000C05D179990476D1C7F1C4F45F6DBE003C5
:107BB0000CD553462146179A039800F095F90544D1
:107BC00004E030205246179990476D1C0099481EDA
:107BD00000900029F5DC08E00298029952460078EE
:107BE000491C0291179990476D1CBBF10001ABF144
:107BF000010BF1DC5BE100F065F90544761C30789F
:107C000000287FF40DAE19B02846BDE8F08F0000C3
:107C10000928010030313233343536373839616262
:107C20006364656600000000303132333435363726
:107C3000383941424344454600000000600700D403
:107C4000062708F1070020F00700F0E8022380462D
:107C500003F0004C5FEA0C0001D097A009E020057A
:107C600001D596A005E0E00701D095A001E0AFF2B4
:107C70004C001390307823F0004365280CD006DCCC
:107C8000452809D046281DD047287FD13BE06628EB
:107C900018D067287AD136E00021112F01DB11209E
:107CA00000E0781CCDE9000104A90CA8FFF7EEFC68
:107CB000DDE90D010C9A4FF0000B07F1010910925C
:107CC00000914EE04FF000400097CDE9011004A96B
:107CD0000CA8FFF7DBFCDDE90D020C9B0F994FF0C0
:107CE000000B91461093009211B9791C00EB010929
:107CF000B7EB090003D4C0F1FF3B07F10109A9EB81
:107D00000700019042E0012F00DA01270021112F26
:107D100001DD112000E03846CDE9000104A90CA8DE
:107D2000FFF7B4FCDDE90D010C9A00914FF0000B58
:107D3000B946109221070FD4009A4A4503DA9146BA
:107D400001E0A9F10109B9F1010F05DD109AA9F1CE
:107D50000101515C3029F4D0B84202DA10F1040F6D
:107D600003DA0121CDE9011010E0002803DC83448F
:107D7000A9EB000102E0411C494500DD8946A0EB6A
:107D80000B00401C01904FF000400290200705D4EA
:107D90000198484502DB4FF0FF30019000208DF83C
:107DA0004B0002980DF14B07B0F1004F25D0022097
:107DB0000C902B200D90029800280CDA4042029083
:107DC0002D200D9007E00A210298F8F70BFD3031C5
:107DD000029007F8011D0C99481E0C900029F2DC56
:107DE00002980028EFD1791E0D980870307800F0C5
:107DF000200040F0450007F8020D11A8C01BC01D6F
:107E000002901398007800B1012000EB090101985D
:107E100001EBE071029801440398401A401E039060
:107E2000E00306D453462146179A039800F05CF805
:107E300005441398007818B15246179990476D1C65
:107E4000E00323D553462146179A039800F04CF8D7
:107E500005441BE0BBF1000F07DB0098584504DD2B
:107E60001098179910F80B0001E01799302052462E
:107E7000904701980BF1010B401E05F1010501909F
:107E800004D12E205246179990476D1CB9F100017C
:107E9000A9F10109DEDC05E017F8010B524617993C
:107EA00090476D1C0299481E02900029F4DC53464D
:107EB0002146179A03989EE62D0000002B00000033
:107EC000200000002DE9F041044600251E4617461B
:107ED000880404D405E039462020B0476D1C641E98
:107EE000F9D52846BDE8F0812DE9F041044600258A
:107EF0001E469046C80301D5302700E0202788049D
:107F000004D505E041463846B0476D1C641EF9D5DE
:107F10002846BDE8F0810A68531C0B60107070475A
:107F200010B504462CB1FDF735FE01200549087057
:107F300010BD0020F9F772F900200249087000BF57
:107F4000F6E70000EC01002013B50C464FF47A73FD
:107F5000012269460248FCF7B3F900981CBD0000F5
:107F600020040020FAF796FEFEF7E2F9FDF7C4FBC5
:107F7000FDF7A6FBFDF778FDFDF792FDFDF708FD87
:107F8000FDF796FCFDF72AFDFDF744FBFDF74CFDE0
:107F9000FDF770FCFDF7C4FC00202E4908602E4957
:107FA00008602E490860002210212D48FAF7F8FADF
:107FB000F9F718F8FCF7AEFCFCF752FDF9F702FAF6
:107FC000FDF7D6FD27A0FFF775F8FDF7D1FD0020DE
:107FD0002C4908702C490860FDF782FD2BA0FFF7A3
:107FE00069F83648FBF7DAFB3548FBF7D7FB35482D
:107FF000FBF7D4FB3448FBF7D1FB2AE0FCF7FEFD8E
:10800000F9F714F83148007801280CD0022807D07D
:10801000032802D004280CD108E0F9F705FA0CE097
:10802000FDF71AFA09E0F9F70BFB06E0FDF772FF1E
:1080300003E003202549087000BF00BF24480078F2
:1080400020B1FEF7B3FE0020214908700A20FAF79C
:1080500091F9D3E704020020080200200C0200205E
:1080600000180240496E697469616C697A696E67CB
:10807000206F7A6F6E6520636F6E74726F6C2E2E38
:108080002E0A000040010020440100204F7A6F6E4C
:108090006520696E697469616C697A65642C207702
:1080A000616974696E6720666F722072656D6F74A6
:1080B0006520636F6E74726F6C0A000048030020C5
:1080C00090030020B80200200003002018010020C7
:1080D00050000020000610160006101600000000D8
:1080E0000000000001020304060708090000000068
:1080F000010203040000000004FA97999999D93FFE
:10810000AF788E1DC571CC3F9FC678D0099AC33F0A
:10811000935555555555E53F599322942449D23FDF
:10812000DE03CB966446C73F44523EDF12F1C23FA6
:108130000000000000000000DDDDDDDDDCBBBBDD9C
:10814000DDDDDDDDDDDDDDDD9888888888888888F7
:108150007777777777888888855555566666666617
:1081600066666666666888888333333222222222F6
:10817000222222222228888D7B225834223A25640A
:108180002C22583130223A25642C22583132223A9E
:1081900025642C22583133223A25642C225831345C
:1081A000223A25642C22583135223A25642C225853
:1081B0003138223A25642C22583230223A25642C58
:1081C00022583231223A25642C225835223A252E63
:1081D00032662C22583232223A252E31662C225811
:1081E0003233223A252E31662C22583234223A2557
:1081F000642C22583235223A25642C2258333522F9
:108200003A25642C22583337223A25642C225833DD
:1082100038223A25642C22583434223A25642C2200
:10822000583436223A25642C22583437223A2564B1
:108230002C22583439223A25642C22583530223ADF
:1082400025642C22583531223A25642C22583532A7
:10825000223A25642C22583533223A25642C2258A0
:108260003534223A25642C22583535223A25642C9F
:1082700022583536223A25642C22583537223A25A1
:10828000642C22583538223A25642C225833303059
:10829000223A252E36667D00B882000800000020B4
:1082A0001C0200002C0E0008008300081C020020A5
:1082B000440F000070760008012C32104201035D6B
:1082C00024F45A03685A020C2904290CA9046924CD
:1082D0009A042029106930A94009120C9A093469BE
:1082E0000C01194A01F7390B19010914234904E15A
:1082F0002370411AA004091657016632140233286C
:040000050800018965
:00000001FF
